:020000041100E9
:10300000002373B52B4D2C4C28006361022601F080
:103010006BF94021FE2221742800284B009601F014
:10302000B5F9002836D1217CFF222800244B0096D8
:1030300001F0ACF900282DD1224BA2899A4226D169
:10304000E389214A93420DD1204B6361204B2268D2
:10305000002A03D1002B01D043CB43C4280001F048
:1030600081F973BD1B4A934201D00023EFE71A4B4D
:103070001A4A1B68934206D9C02304222800217CE7
:103080009B0001F0F9F9114B6361154BDFE7002359
:103090002374EAE7CC233821AC2228009B01217459
:1030A00001F0EAF90028F2D10E4B63610E4BE38187
:1030B0000E4BCCE7AC42FF1F7C62FF1F8862FF1FF4
:1030C0008A62FF1F59590000830500001541001155
:1030D00068BD001182150000A062FF1F8713000069
:1030E00074BD0011CD410011AAAAFFFF5CBD001103
:1030F000F7B5164B0192C318021D002000938823D8
:103100005B05D3181B685C1C1AD09CB2402C18D8E5
:103110008D781E0CAC466746CD782D023D43AE42FD
:1031200006D1019800280ED110000C70240A4C70B2
:1031300003249BB20733A343D218009B9A42DED3E9
:10314000FEBD4432F9E71000FAE7C046FC0F00006C
:10315000802213B503000324019189B25201073183
:103160009B18A14304305A1A88235B05C3181B68B7
:10317000591C03D190429241104016BD99B240298A
:1031800007D80B000733A343C0189042ECD30020AC
:10319000F3E74430F9E7134B134A1B68126810B584
:1031A000FA24934201D81A00F824104BE4021B6859
:1031B0009A4210D813000E4A12689A420ED3013375
:1031C00007D1F823DB029C4203D10A49054808F0E5
:1031D0005FFB200010BDFC24E402ECE7FE24E402C7
:1031E000F7E7C04600C0071100D0071100E0071143
:1031F00000F00711FFFFFF7FF0B59BB015000490B2
:103200000391402A00D9A0E006AB59801A80FFF74D
:10321000C2FF0400042816D9002206A9FFF768FFA0
:10322000052810D906AB1B88AB420CD1002D07D066
:10323000514B2A000499C01808F0FAFA002802D16C
:1032400001201BB0F0BD06AB1D8020000699FFF7E2
:103250007FFF041E7BD1069B0793FFF79CFF802313
:103260005B01C618802307001B039E4201D3F8268A
:10327000F60288235B05F31801931B68013302D023
:10328000019808F045FB3D49019808F001FB3B1D02
:103290000293331D05938822029B52059B181B68DD
:1032A00008935A1C3CD044219AB20091402A04D879
:1032B0000320D11D814389B2009103991B0C8B42DD
:1032C00024D0402A22D80122300008A9FFF710FF9D
:1032D000021E1BD1380008A9FFF70AFF04000428CA
:1032E00031D9009A059B9B1880225201B218934253
:1032F00040D288235B05C118009A09A808F070FA2B
:103300001D4B009A09A9F01808F0F2FA009A029BE6
:103310009446634402931A4B029AFB189A42BAD31A
:1033200088235B05FC1821680198013908F0B0FA80
:10333000200008F0EDFA039A07AB5A803000079995
:10334000FFF706FF0400002C03D1002079E70428D2
:10335000FBD988235B05E018069908F099FA032346
:10336000EA1C9A4300D16BE7034B0499E01808F07C
:10337000BFFA65E70424ECE704000011FFFFFF7FBC
:10338000F80F0000F7B505001400402A21D80027E7
:1033900001AE71803780FFF7FEFE042816D93A008F
:1033A0003100FFF7A5FE042810D93688BC420BD0A7
:1033B000BD4209D0221CB44200D9321C064B92B245
:1033C000C118280008F00CFA30B2FEBDC04300B2AC
:1033D000FBE703204042F8E70400001137B5042260
:1033E00004000D0001A81649FFF7CCFF02000428D5
:1033F0000BD1019BA34208D3AB4204D0104901A8D2
:103400000195FFF7F9FE01203EBD0E4C2368200018
:10341000019308F07DFA019920000139019108F02B
:1034200037FA80235B01E418074B9C42EED104225B
:10343000034901A80195FFF7DFFE0020E4E7C0463D
:103440005555000000C007110000081130B589B0C3
:1034500008F00EFA10226946254808F029FB254B92
:10346000009A9A420ED1019B029A0F2B33D8002169
:1034700001240698013B08D2002900D00292029B49
:10348000013331D10023029325E0551CF2D1020013
:103490002100EFE710341022200004A908F008FBF7
:1034A000029B013301D1069B0293882304995B059B
:1034B000C918059B06981A03120B049105928142C4
:1034C00003D02B4201D108F08BF9019B013B019302
:1034D000019B002BDED1029B002B03D004930498A8
:1034E0004168084709B030BDE025014C2D03EFE7E6
:1034F00000000111504859368022F8B5964C974B80
:10350000D200002120001C6008F07AFB2300944ABE
:1035100088331A60934B1A786A23002A00D011333B
:10352000E3620A232365904B37221B780820A363AC
:103530008E4B2118E361102323628D4B3B25636181
:10354000C823DB00A36123008C331A602823013ACF
:10355000E26320646364CA67043A211DCA672100DC
:10356000BC310D602100C03108602100C4310B6006
:1035700021000635CC310D602100083DC8310D60B9
:103580002100D0310A602200D43210602200D832EB
:10359000136022000227E032210017604222DC3152
:1035A0000A6021001B3DE4310D602100E831086014
:1035B0002100EC310B6023000521F4331960230056
:1035C000F0331A602300183290331A6023009433CA
:1035D000186023001E3A98331A60AF23DB00236083
:1035E000644BFA262363644B644DE360644BF03113
:1035F000A3642300FF31FC33B600A16021611E608B
:10360000A5627325E5656D3D6565A56596255D4AF1
:10361000AD00E264666258606766A566002709250A
:10362000A767E566584F594D606720002567E26738
:103630003A6015279C30676007001A203860200028
:10364000A0300700212038602000A83007004C4837
:1036500038602000F830066026006427A436376002
:1036600026005F3FAC3637602600033FB036376038
:103670002600C637B436376026000027B8363760D4
:1036800038269E60424E96205E64424E5A66DE6147
:10369000414E9A645E62F53EFF3E9E621E269A6728
:1036A000354A8000DE661F675F67DD651D6618624C
:1036B000DA67BE23394A5B00E250394BD8382350D1
:1036C00004302250C4225200A350C623E4205B00E1
:1036D000E1500433334AE1503349344BD16034492B
:1036E000800019503349E938FF3819503249043005
:1036F000195032493248D16132491163324951631C
:103700001900F4310860CE20304940001160304982
:10371000195019002F48F83108602F49D1658221CE
:103720002E4A89005A501A002D490832D1671A00D2
:103730002C49B432116088212B4A89005A501A0052
:103740002A49883211602A4ADA6408F0D9F801203F
:1037500008F006F8F8BDC0460004FF1F2065FF1FF3
:103760000070FF1FEC44FF1F4A0AFF1F3A070000CA
:1037700080C3C9019A020000DC0500006A1800003D
:1037800050C3000088130000F009FF1F204E000006
:103790006509FF1F68100000C409000040420F00C7
:1037A00010270000FC00FF1F7D1CFF1F0000FF1FF3
:1037B000D12CFF1F6130FF1FF92EFF1F3D20FF1F7F
:1037C0002D27FF1F5920FF1F0522FF1FC91FFF1FA5
:1037D0005129FF1F392AFF1F9519FF1F5D28FF1F61
:1037E0008125FF1F8D25FF1FC91EFF1F811FFF1F82
:1037F000411EFF1FF0B502250124604B91B01D70E2
:1038000002935F4B5F4E1C705F4F03933368002140
:103810002800FB7006F018FE280006F00FFD0023BC
:10382000984205D0FA78552A02D0332A00D098E081
:103830003360042006F070FF07F0F2FEFFF75CFE35
:1038400008F006F91F2201240021504B10AD1A7018
:103850004F4B1C704F4B19704F4B19689143163AE0
:103860000A431A60602219689143403A0A431A6079
:1038700008F0E6F908F0B4F9C120FF21474B8000B9
:103880001A588A431A50C522920098588843BF3963
:10389000014399509858424908408021C901014389
:1038A000802099509958C0050902090A014399508E
:1038B00080213C48490108F07BF8032322003A4963
:1038C00001940093394808F003F82C22384905A8E0
:1038D00007F086FF05AC61782078023406F0CEFC54
:1038E000A542F8D1334C344B226803201A40A02360
:1038F000DB0213432360802322689B04134323606D
:1039000022682E4B1A4080239B03134323602C4ACA
:103910002C4B934200D8012008F0DAF808F078F92F
:1039200080232268DB0413432360029B187808F08D
:103930000FF9039B1878C0B208F062F808F070F82D
:103940002149042008F0E4F806F0B2FE00F03EF849
:1039500000F0E8FD00F090FE00F00AFA002011B03F
:10396000F0BD00932100184A042008F0E1F88023FC
:10397000DB059C62FFF76AFD5BE7C0464A0AFF1F52
:10398000EC44FF1F34F00040AC62FF1F480AFF1FE9
:10399000490AFF1F680AFF1FBCF0004000E100E079
:1039A000FF00FFFFF044FF1F7457FF1FF054FF1F7D
:1039B00080BC001114F00040FF7FF8FFFFFF9FFF65
:1039C0000080FF1F0070FF1F3B000108002210B5A0
:1039D0001100112007F034FE10BD0000F8B50023DF
:1039E0000925374F374C3B62E3681120AB43E36056
:1039F00007F006FF112008F0B3F8112007F0C0FE11
:103A00004023226880261343236080236268DB0200
:103A100013436360A3682C4A3343A360A368280060
:103A20001340A3608023A2689B0113431022A3606C
:103A3000236C022193432364236C0F3A13432364C2
:103A400080235B013B62226B204B1A402263626B36
:103A50001A406263A26B1A40A263E26B1340E363F5
:103A6000E3681B4A1340E36006F008FC28000121CC
:103A700006F018FD8023174A9B00516C11200B4360
:103A8000536407F065FFFD21134B144A89005A5017
:103A90008023C720E26B5B031343E363E36880008A
:103AA0001D430F4BE56019580E4A11408022120247
:103AB0000A431A50802292051A600B4B5E63F8BDD0
:103AC00000F000403CF00040FFFFDFFFEFFFEFFFA2
:103AD000FFFF7FFF003800400000FF1F5118FF1F4D
:103AE00000E100E0FF00FFFF0000054070B5284C3A
:103AF000238C002B23D0228A002A21D1DA002382B2
:103B00006382A382E38223836383A383E3832260AC
:103B10006260A260E2601F4D1F4A6420EB80934206
:103B20000AD8FA220020D200934205D91B4A0A2162
:103B3000981807F02DFFC0B200232872238470BDAF
:103B40000720E11CCA7F01320240CA7705D1032554
:103B5000201DC17F01312940C17708325200A35294
:103B6000002321001A00088A01321B180231082A9A
:103B7000F9D1221DD27F9200A350626823689B185E
:103B8000A2689B18E2689B185B099BB2C3E7C0461A
:103B9000EC61FF1F9462FF1FB70B000030F8FFFFBE
:103BA00030B503A804880B20002C0ED14968074DBE
:103BB00008784978090201430A20A94205D1012168
:103BC00020001980024B1B7A137030BD192A0000A7
:103BD0009462FF1FF7B5150008AA16884A680F4FB0
:103BE00014785278120222430A24BA4214D10122D4
:103BF000DBB2019200962A0007F0AAFC041E0BD14A
:103C0000074B1B68002B07D068782A780002104306
:103C100042425041013098472000FEBD0229000079
:103C20001862FF1F30B5012503790400BFB02B4295
:103C300011D00A49408806F0F7FF28420BD0084B04
:103C400001A95B8D4D800B80064B00221B7A60889A
:103C50000B7104F0DBF83FB030BDC0461062FF1FAF
:103C60002041FF1F9462FF1F10B50549054806F06B
:103C700091FF0421044A054806F04EFF10BDC046DE
:103C80001062FF1FFFFF0000ACBC00112041FF1FAE
:103C900010B5024804F03CFF10BDC046253C0011A1
:103CA000012303700B4B1A7A4270022282709A78B9
:103CB000C270DA780271032242711A7982715A79DC
:103CC000C2710C2202729A794272DB7983720B20E4
:103CD0007047C0469462FF1F022310B50370013B7A
:103CE00043700533837010330371443B43712A33AF
:103CF00083714433C37100230372064B04001B8895
:103D000043720A30FFF7CCFF831D0A30C0B2E37064
:103D100010BDC0469462FF1F10B5142007F0E0FCF0
:103D2000124B14220021186007F06AFF002007F0F0
:103D300037FF012007F0D4FD022007F051FE0320D9
:103D400004F08AF9042006F09FF9052003F0C8FB6F
:103D5000062004F095F8072001F05EFA082006F02E
:103D6000BBFE092001F038F810BDC0461C62FF1FE1
:103D700007F0C6FC012007F07BFC07F0C9FC00003F
:103D8000094B10B50400984205D0012904D1200048
:103D9000064906F0FFFE10BD0229FCD1013904F0EE
:103DA00075FE0028F3D0F6E7FEFF00004262FF1F19
:103DB00070B50D7A100004AA2C0016881022144049
:103DC000154220D1002E20D10A78022A18D14A6843
:103DD000517815780E4A09022943914205D00D4ABF
:103DE000914209D01C800A2404E014220A491A8056
:103DF00007F0F6FC200070BD0C2208491A80F7E796
:103E00001C800124F6E70824F4E70B24F2E7C046FF
:103E1000F3FF0000F4FF00007843FF1F8CBD00118A
:103E200010B504000749084806F0B4FE074804F03E
:103E3000AFFD0020E40704D50721054A054806F038
:103E40006BFE10BD4262FF1FFFFF0000813D0011AD
:103E5000F0BC00116441FF1F00B50C4BBFB01A78D5
:103E60000B4902A800F0C2FC6B4680B2D880002843
:103E700009D06A46074B01A91B889380064B002294
:103E8000188803F0C3FF3FB000BDC0462062FF1F8B
:103E90002162FF1FBE41FF1FC842FF1F00B50C4B30
:103EA000BFB01A780B4902A801F0F6FE6B4680B24B
:103EB000D880002809D06A46074B01A95B8D938002
:103EC000064B0022188803F0A1FF3FB000BDC0469A
:103ED0004A62FF1F4B62FF1F6441FF1FC842FF1F62
:103EE000F7B50E00377A1C0008AB11003D001A88A8
:103EF00020231D401F423CD13378022B3BD17368F5
:103F00001F785B781B023B431E4FBB4208D01E4FFD
:103F1000BB4214D01D4DAB4221D00A252800FEBD66
:103F2000002A2AD1142C2AD82200F06807F058FC65
:103F3000174B1C70012CF1D9FFF7B0FFEEE7002AF8
:103F40001BD1202C1BD82200F06807F049FC114B34
:103F500004211C70104B187807F09AFDDEE7E3B2DD
:103F60000124009201940A00310007F0F1FA0500E3
:103F7000D4E70825D2E70125D0E70B25CEE70D25AC
:103F8000CCE7C046F3FF0000F4FF00000229000068
:103F90004A62FF1F2062FF1FCC62FF1F332310B550
:103FA000040003700A220749013007F019FC064B90
:103FB0000F201B681A0AE37222731A0C1B0E62731D
:103FC000A37310BD9462FF1FBC62FF1F30B50125B3
:103FD00003790400BFB02B4213D00B49408806F090
:103FE00023FE28420DD06A46084B02A81B88938006
:103FF000FFF7D4FF6B46D8800022608801A903F048
:1040000005FF3FB030BDC0464262FF1FBE41FF1FEB
:1040100010B5024804F07CFD10BDC046CD3F001134
:1040200070B5160004AA148805AA15784A68507855
:10403000117800022A4A0843801805284BD807F057
:10404000B7FD03131E29343F0720042C0BD805228B
:10405000121BAA4200D92A0022491A8030000919ED
:1040600007F0BEFB002070BD0720112CFBD81222E8
:10407000121BAA4200D92A001B491A80EEE707202A
:104080000E2CF0D80F22121BAA4200D92A00174981
:104090001A80E3E70720032CE5D80422121BAA426A
:1040A00000D92A0012491A80D8E70720032CDAD851
:1040B0000422121BAA4200D92A000E491A80CDE719
:1040C0000720032CCFD80422121BAA4200D92A00B1
:1040D00009491A80C2E700220A201A80C3E7C046B5
:1040E000DCD5FFFF3BBD00116862FF1F2BBD001137
:1040F00026BD001121BD00111CBD001110B50D2100
:10410000024A034806F008FD10BDC04610BD00116C
:10411000D441FF1FF0B50024274E85B03000B471A4
:1041200000F0E2F8254D264BEA89297C9A422FD1EE
:104130000423300003AA00F057F90400300000F017
:1041400011F90123B371002C34D16B4699892B6886
:10415000C9BA4B4329891B4A1B145B1853806B4611
:10416000D9896B6849BA89B24B4369891B0C5B18C2
:104170001548191C1BB2834200DD011C0B0400D53D
:1041800000211388918001331380200005B0F0BD19
:104190000227220003AB3000009700F0F7F80E234F
:1041A0000400297C0122300000976B4400F0EEF8F7
:1041B0000443C3E71C00E8E7AC42FF1F7C62FF1F1B
:1041C000830500009462FF1F0F27000073B5234E84
:1041D000300000F089F8224D07236A463000297C20
:1041E00000F002F904003000002C33D16B461B783C
:1041F0007F2B2FD800F0B6F86B46D878F023020456
:104200001B031A406B469B8816495BBA9BB21A4344
:104210002B68000953432A891B0C9B184B806B4663
:104220005A789B7812031B011A436B68024353436D
:104230006A891B0C9B180C481A1C1BB2834200DDB8
:10424000021C130400D500220B888A8001330B80E6
:10425000200076BD00F086F80124F9E7AC42FF1F8C
:104260007C62FF1F9462FF1F0F27000070B5114C86
:10427000237C002B0FD0382B0ED10F4D280000F0DF
:1042800033F8CC23AC222800217C9B0100F0F4F809
:10429000280000F067F870BD084BE2899A42FAD115
:1042A000054D280000F020F800222800217C00F0B5
:1042B000C5F8EDE77C62FF1FAC42FF1F83050000DD
:1042C00010B5084B1A7C002A09D05B69002B06D078
:1042D0009847041E01D0FEF793FE200010BD012474
:1042E000F9E7C0467C62FF1F70B5C17905000C007C
:1042F000631E9C411A4BE402E41849000460C9B2F1
:10430000007906F005F9E979687949000131C9B207
:1043100006F0FEF8E8790930C0B207F031FA002360
:10432000E36661332360AA795B3B002A0ED02268E2
:104330009A43023B134323600A23E361073323625A
:1043400000232363A3630133E36370BD22689A43B0
:10435000022313432360462363610633A361EFE71F
:104360000050004070B5002504000368DD66C07988
:104370000930C0B207F044FA2900207906F064F849
:104380002900607906F060F870BD0000F8B51E00E5
:1043900006AB1D78002304681700E366616007F030
:1043A00067FA01238022E3662B0027615200013B5C
:1043B00008D207F0DDFA08200A4A1168002D03D15F
:1043C0002800F8BD2261F2E7236F034203D023697E
:1043D000013D3370013613685B1A032BEED90125BA
:1043E000EEE7C0466008FF1F70B51C00002305689B
:1043F0001600EB66696007F03BFA01238022EB664A
:1044000023005200013B08D207F0B2FA08200A4A02
:104410001168002C03D1200070BD2A61F2E72B6FD8
:10442000034203D02B69013C3370013613685B1AD9
:10443000032BEED90124EEE76008FF1F002370B5BF
:1044400004681500E366616007F012FA0123E36671
:10445000256107F08DFA8020064A80001168636BA1
:10446000034205D113685B1A032BF8D9012070BDF4
:104470000020FCE76008FF1F70B51D0000230468E2
:104480001600E366616007F0F3F90123E366266135
:104490000F33626B1A42FCD02B0A23611023626B2C
:1044A0001A42FCD0EDB2256107F062FA8020074A7B
:1044B00080001168636B034205D113685B1A032BFC
:1044C000F8D9012070BD0020FCE7C0466008FF1F3E
:1044D00070B51E00002305681400EB66696007F0E4
:1044E000C7F90123A619EB660F33B4420ED107F0CA
:1044F0003FFA80200A4A800011686B6B03420CD19E
:1045000013685B1A032BF8D9012070BD217829614B
:10451000696B1942FCD00134E7E70020F5E7C0469B
:104520006008FF1F10B5084CE368002B08D18022FB
:10453000064B52021B689B186360054B1B68236087
:1045400007F086F8A06010BDBC62FF1FC8F00040F5
:10455000CCF0004070B5184A936A916A9942FBD139
:1045600016498A689A421FD39A1A8B60144B012607
:10457000186893B2D202D20E4343424300204C68E3
:104580001B0A1B1912029B180E4C0A684B60551C23
:10459000A3420CD8002801D04B600A600A4A13607D
:1045A00008680A4B186070BD581E821ADDE7084A79
:1045B00030009B182A00EAE700F00040BC62FF1FB1
:1045C000140AFF1F40420F00C8F00040CCF000402A
:1045D000C0BDF0FF70B51F4C23793F2B01D93F239D
:1045E00023711D4B22791A701878C0B207F030FB86
:1045F00018231A491A4A0B801A4913800B805380DA
:10460000A379194980200B800C21938001334B43FF
:10461000164D191C0001834200D9011C2980D1804C
:104620006379002B11D101336371237A012B01D8F7
:10463000022323726279237A0D4853430A21584397
:1046400007F0A6F90B4D286070BDA02BEDD9A02373
:10465000EAE7C046B062FF1F480AFF1FC642FF1FBD
:104660009844FF1FC442FF1FC242FF1FC042FF1FEA
:1046700071020000A062FF1FF8B514210020FEF7B0
:10468000ADFE114C011E114D09D10C22104BC1CBB6
:10469000C1C4280007F0B4FAFFF79CFFF8BD0C2254
:1046A00020000C49FEF76EFE0C2802D0084B43CBCD
:1046B00043C40C2228000849FEF764FE0C28EBD006
:1046C0000C220021E5E7C046B062FF1F7C62FF1F9D
:1046D00080BD0011FC0C0000F50C0000F0B51D4C75
:1046E0008022A5440400882069465201400507F055
:1046F00037F9902212016A441300200032C832C3F5
:1047000016C816C38023144C144FA6689B0333436A
:10471000A3603B6007F0C4F98823A0685B05C0185C
:1047200007F0F6F80025882329008022A0685B05A1
:10473000C01840196944520007F0DAF880230135A7
:10474000FF355B019D42EED1A6603E60044B9D4467
:10475000F0BDC046FCEFFFFF0844FF1F9808FF1F95
:1047600004100000F0B5040087B0002825D068468A
:1047700006F076FF1B4C022806D10622694620006F
:1047800007F056F8002816D06946002301250F26A9
:104790002F00E25C013310091030874038002F00F1
:1047A000324097403A0002434A610439062BEFD168
:1047B0006846FFF793FF07B0F0BD182269460A4824
:1047C00007F0CEF86A46A300D358013305D018226B
:1047D000FF21684607F014FAEAE70134062CF1D10C
:1047E000E9E7C0466509FF1F00090011F0B5002583
:1047F00004000E0085B0AA4200D186E04B1C087868
:1048000001934B788978377909021943F3783F0689
:104810001B040B431F43039720706570252800D1AC
:1048200096E033D8112813D807F022F9690028013F
:10483000280128012801AA00B800B1002801280198
:10484000280128012801280128012801020122014C
:10485000232800D1DBE0DB2800D031E1042A00D896
:10486000ACE01025052A05D0551F2A003800711D1F
:1048700006F0B6FF05223100200006F0B1FF2A0045
:104880003900601D06F0ACFF05353EE0562859D0D2
:1048900010D8332800D19DE0552839D02628DAD108
:1048A0009D4B2900132218001D0007F0A9F9FEF7FF
:1048B000A7FB5CE0712800D177E0722800D180E08E
:1048C000602800D18BE0DC28C5D1022A00D875E031
:1048D0007378BFB26370B378A370032A05D0033A2C
:1048E000390092B2F01CFEF787FC10223900E01C60
:1048F000FEF748FDC51C002807DA60705CE00C225A
:104900002000864906F06CFF0C25280005B0F0BD9C
:10491000013A834D0C2A13D8002A0AD028000199A5
:1049200006F05EFFFFF756FE0C2228007D49FEF7D9
:1049300063FC29000C22601C06F052FF0D25E4E701
:104940000C22EBE7764D784B2A0043CB43C2E9E7D4
:10495000013A714D0C2A11D8002A08D0019928007B
:1049600006F03EFF0C2228007049FEF745FC2900A6
:104970001322601C06F034FF1425C6E70C22EDE775
:1049800005226B49601C06F02BFF0625BDE71222AD
:104990006849601C06F024FF1325B6E70822664923
:1049A000601C06F01DFF0925AFE77178F02905D8D6
:1049B000624B188801F0CCFD0225A6E7FF23637047
:1049C000FAE75F4B012A03D072789A706270F3E7BE
:1049D0009B78F4E72000FFF7E1FA050095E7013A3C
:1049E000574B584D082A0DD8002A0DD00121280018
:1049F0005970019906F0F4FE01F082F808222900AE
:104A0000601CCEE70822F1E700225A70F6E7042A7C
:104A100004D94D4D2F6006F01BFEA860FFF79AFDEC
:104A20000422039003A9601C06F0DAFE05256CE75A
:104A3000464D062A15D906222800019906F0F8FEEF
:104A400000280ED006220199280006F0C9FE062291
:104A50003F492800FEF7D0FB0123394A91780B43E8
:104A6000937029000622601C06F0BAFE07254CE769
:104A7000012AA3D07078FFF775FE9DE7012800D0CA
:104A8000E9E6931E334F132B04D87378002B09D11A
:104A900000F014F9304B39001D78601C6A1E06F0D6
:104AA0009FFE32E7551E2A000199380006F098FE55
:104AB0002A49AAB23800FEF79FFB00F037F9E9E770
:104AC000DA281DD1042A00D878E7082A15D9B37945
:104AD00072791B021343F27912041A43337A1B06CC
:104AE00013433B603B68052231002000039306F02E
:104AF00077FE0422601D03A953E7FE236370F1E7EC
:104B0000DE2800D05AE7511E012A01D10025FCE61B
:104B1000019800F0DBFFF9E77C62FF1F8CBD0011FC
:104B2000B062FF1FFC0C000080BD0011F50C0000FE
:104B30008862FF1F6862FF1F0C44FF1FC842FF1FEF
:104B4000AC62FF1F6543FF1FBC62FF1F6509FF1FAB
:104B5000ADAC0000AD64FF1FAB64FF1FAEDE000014
:104B600070477047020010B5094B0A32094C92B2E7
:104B7000DA815A8298811882207802F04FFB042251
:104B8000054B012120781A7006F082FF10BDC04647
:104B90009643FF1FF664FF1FF564FF1F013870B5D1
:104BA000042809D807F004F8030928081200234B49
:104BB0000221187806F06CFF70BD204B0821187890
:104BC00006F05EFE00221E4B1A72F5E780220024DA
:104BD0001B4B1A4D52001A8108211A682878DC7282
:104BE00006F09EFF2100287806F082FD012000F0EB
:104BF00073FE00F085FFDFE7104B0821187806F000
:104C00003FFE1048FFF768F80F4B104A9B790020D1
:104C100093800F4A13808022094B5200D8721A8168
:104C200000F05AFE00F06CFF0A4B9B78002BC3D0BB
:104C3000094A136006F074FDBEE7C046CC62FF1F50
:104C4000A062FF1FD142FF1FB062FF1F9844FF1FE9
:104C5000C242FF1FAC62FF1F34F0004010B50129B3
:104C60000BD1022809D1054B1B78002B05D0262239
:104C7000034B04485A72FFF775FF10BDCE64FF1F47
:104C8000A062FF1FC40900000300F0B50A4D8E1892
:104C9000B14202D152008018F0BD0C782F6824096F
:104CA0003C5D0F271C700C7801313C402F683C5D47
:104CB0005C700233ECE7C046BC42FF1F0E22124B71
:104CC00010B51A700D23114C11492370093A043B99
:104CD0001048637006F084FD2D2301220E490F4811
:104CE000E371FFF7D1FF01220D49FFF7CDFF01224C
:104CF0000C49FFF7C9FF030000200B4902001870A0
:104D0000FEF77AFA10BDC046CA64FF1FAB64FF1FEE
:104D10003BBD0011AD64FF1F6709FF1FB364FF1F98
:104D20006609FF1F6509FF1FAEDE000070B5124C5B
:104D3000142220001149FEF725FB431E104D132BB2
:104D400017D8AB78002B14D0431C2B7009236B7041
:104D5000002300190370287829000130C0B206F042
:104D600067FC297822000139C9B2002005F0F2FD64
:104D700070BDFFF7A3FFEEE7AD64FF1FAEDE0000DE
:104D8000AB64FF1F10B5114B1A781870002A0ED0B3
:104D900000280BD10E4B1A78062A07D85423D3408B
:104DA000DB0703D50B4B187802F038FA10BD00284A
:104DB000FCD0074B1B78012B02D0033B022BF5D80C
:104DC000044B0121187806F063FEEFE7CE64FF1F65
:104DD000F564FF1FF664FF1F70B54A4E4A4A4B49FF
:104DE0003070022005F042FC00F0F2FEFEF708F9F8
:104DF00006F026FD032246494648FFF745FF2D24CD
:104E0000030004221C7044490130FFF73DFF3023AA
:104E10000470424D424C437083702E3B06222000AA
:104E20004049EB87FEF7AEFA062813D0200006F0C3
:104E300017FC022809D00321200006F0C9FC8D23AD
:104E4000E3706E3B237119336371062220003549EC
:104E5000FEF7D2F9344B1B68FC335C64FFF766FF46
:104E60000020FFF78FFF314C314A0121314B12787E
:104E7000207802F095F9304A304B127800212078E2
:104E800002F08EF901222E4B1A702E4BDB78552B37
:104E900031D12D4B3B325A722C4B2D4AAB81EA81DA
:104EA0002B826A822021307806F0A2FE0120404247
:104EB00005F09CFD0120404205F038FEFFF71EF989
:104EC000FEF7D2FE00F0B2FC01204042FEF7A8FF40
:104ED000012006F0F5FCF02001F01EFB01213078E6
:104EE00006F0D6FD307802F0F5FA1A4806F0B8FE62
:104EF000FEF774FD70BD6422174B5B7953431A00B3
:104F00000A32CBE7CC62FF1F614B00115D4C0011F0
:104F10000C44FF1F6862FF1F8862FF1F9643FF1F3C
:104F20006509FF1FADAC00002065FF1FF664FF1F81
:104F3000F042FF1FD142FF1FCA64FF1FAB64FF1F77
:104F40009C64FF1FAC62FF1FA062FF1FC40900002A
:104F5000CE090000CE62FF1FB062FF1FF8B50A0045
:104F600020230D001A40194263D05E4B1B78002BA2
:104F70005CD0FFF7EFFA5C4B5C4C5D4E9968626861
:104F8000737A8A1ADB039A4202D36160FEF726FD28
:104F9000327A217A531EDBB2994205D1FFF766F9C6
:104FA000002000F0E7FD15E09142F9D300272772B9
:104FB000FFF786F9A37ABB4202D0A772FEF796FDEF
:104FC000012000F0D7FD4B4F3800FEF785FE390079
:104FD00006F0CEFB637A002B25D0013BDBB2637277
:104FE000002B20D1444BDB78552B01D106F098FBE8
:104FF000E37A002B12D00023A27AE3729A4202D005
:10500000A372FEF773FD3D4A3A4F1388380001330F
:105010001380FEF761FE390006F0AAFB6423707965
:105020005843FFF79FFD237A013323722020684005
:10503000F8BD0BB2002B0ADA314B187806F0F0FB02
:10504000002801D006F02CFB80200002EFE70224AC
:10505000214206D0254B01201A72FFF793FE200053
:10506000E5E70B071ED5FFF775FA1F4B1F49204CCC
:1050700098684A68637A821ADB039A4202D34860CE
:10508000FEF7ACFCFFF71CF9FFF7F0F8012000F089
:1050900071FD00F0E5FB2368DB0701D5FEF7B8FFE3
:1050A0000820C4E7CB0609D5FEF720FD0D4B1B7881
:1050B000002B01D1FEF7ECFD1020B8E701242142BE
:1050C00007D0104800F06CF806F0CAFC00F034FD80
:1050D000C5E70424080020402142A9D0FEF7BCFE09
:1050E000BDE7C046CE64FF1FBC62FF1FA062FF1F6A
:1050F000B062FF1FD142FF1FAC62FF1F9462FF1F0F
:10510000CC62FF1FB442FF1FF0B51B4B1B4F1B8827
:105110003A8804001A4E1B4D85B09A420DD8328849
:105120009A420AD3184B1A882B889A4205D1174AFB
:10513000174B12881B889A421BD0052001F042FAB7
:105140003B8802AA13803388019053802B88114D2D
:1051500093800F4B02A91B88D3800F4B2A781888A5
:1051600002F05EFF0D4B08212878019A1C7006F0B2
:10517000DFFA05B0F0BDC0469A64FF1FC642FF1FAC
:10518000C442FF1FC242FF1F9864FF1F9664FF1FA7
:10519000C042FF1FF664FF1FC842FF1F9464FF1F39
:1051A00013B50C4B1C78002C11D1002801D00A4BF0
:1051B00018600A4A0A4B11780A4A10780A4A019282
:1051C0000A4A0092002205F0BDFA200016BD112403
:1051D000FBE7C046F564FF1F9064FF1FF464FF1FE8
:1051E000E464FF1FF664FF1FD064FF1FD464FF1F39
:1051F00010B5064B12201B78052B06D1044B132249
:105200001988044B187801F0B9FB10BDF564FF1F35
:10521000C842FF1FF664FF1F10B500240122114B86
:1052200052421870104B1C70104B1A8002F052F949
:1052300004220F4B21001A700E480C3206F0D8FBE6
:10524000102221000C4806F0D3FB07220B4B1C60F8
:105250000B4B1C700B4B1C700B4B1A700B4B1C70C8
:1052600010BDC046F664FF1FF564FF1FC842FF1F54
:10527000F464FF1FE464FF1FD464FF1FD064FF1FAA
:10528000AA64FF1FA964FF1FCA42FF1FA864FF1F73
:10529000F8B5174C0600257806A814240078052DCB
:1052A00023D1B41F134FA5B21824BD421DD88D1FA2
:1052B000ADB2BD4219D8FA256D00AA4215D21D0023
:1052C0000D4F0A3DADB2BD420FD80C4C26800C4CA0
:1052D00021800C4900240A800B4A1380FFF714FF39
:1052E0000A4B0421187806F0CBFA2000F8BDC0461E
:1052F000F564FF1F790C0000750C0000C642FF1F0B
:10530000C442FF1FC242FF1FC042FF1FF664FF1FBF
:10531000F0B50BB20D0089B0002B00DB70E1A44E9C
:10532000307806F07DFA041E50D00378A22B00D10D
:1053300022E1D02B1AD0912B45D143780E2B42D1AC
:105340009C4B82889A423ED19B4A83681278052AF8
:1053500039D1032018567F2835D0984B1B68002B75
:1053600031D05B68002B2ED098472CE0807807283E
:1053700029D806F01DFC0428183F3F74A8D863788C
:10538000002B0CD101218C4B19708D4B1A78002AFF
:105390005BD08C4B307801F003FF002855D00722FA
:1053A000854B1A7051E061780029F8D1E378002B21
:1053B00011D0854A854B1278307801F0F1FE60708B
:1053C0006378002BEBD1200006F06AF98020000200
:1053D000684009B0F0BD784B1B78022BF3D0012157
:1053E000307806F0EDF90028EAD10121307806F096
:1053F0004FFBE5E76378002BD1D16F4F032807D12E
:105400003B78052B02D101333B701EE00223FBE702
:105410006F4B1A886F4B0293002A0BD01B78002B1E
:1054200003D00121307806F083F93B78062B04D1B4
:10543000013BE9E7029B1A70F7E7042B41D10121F8
:10544000029B3078197006F023FB5C4B1B68002B25
:10545000B9D01B68002BB6D0574A107884E7637820
:10546000554F002B27D10622211D5B4806F0B8F9C5
:1054700062895A4B5A491A80A2895A4B1A80E38989
:105480000B800521397058490A80584A1380228AB6
:10549000574B1A80574B1B78012B09D11F2001F065
:1054A00091F8FA22920042430421307806F040F944
:1054B0000022484B75E7312B00D070E70022454BA6
:1054C0001A700323A0E706220021434806F090FA51
:1054D0000023454A04211380444A30781380444A0B
:1054E000138006F0CDF90821307806F0C9F9A379C8
:1054F000083B5A425341304A03331370304B1B78F8
:10550000002B06D0334B30781A78002A06D001F0F1
:1055100085FE0122314B52421A8096E70121197013
:1055200006F0B6FAF5E70821307806F0A9F96378B5
:10553000002B00D047E72C4B2D4F0293E388029AB3
:1055400004211380294B307803932389039A138015
:1055500063893B8006F034F9002800D033E7264BFE
:105560001B68002B00D12EE7039902983A8809881E
:1055700000881B68984726E74379132B00D022E761
:105580000389012B0AD11D4B1B78022B06D1082160
:10559000307806F075F9FFF72BFE14E7052001F0CF
:1055A00011F808210200307806F0C2F80BE7C04677
:1055B000F664FF1F05140000F564FF1F9064FF1FD1
:1055C000F042FF1FD142FF1FCA64FF1FAB64FF1FE1
:1055D000CC64FF1FCE64FF1F9D64FF1FC842FF1FE6
:1055E000A464FF1FA664FF1F9A64FF1F9864FF1F37
:1055F0009664FF1F9C64FF1F8C64FF1F9464FF1F51
:105600008020C001014200D0E2E6CB0731D5324B09
:105610001B78002B1DD0314E05AC3378052B1AD1E9
:10562000023B23702E4B21001B7823722D4B1B78DD
:1056300063722D4B187801F057FD002809D0072020
:105640002A4B30701B68002B03D01B68002B00D046
:1056500098470120BCE60E20254B06221B782549E1
:105660002370254B1B78637002ABC01806F0B8F8A6
:10567000D8E7022308001840194209D0174B1B78BD
:10568000052B03D11D4B188806F03AFA02209FE63D
:105690000424214203D0FFF737FD200098E60823B9
:1056A00008001840194200D193E6154B1C78012CD4
:1056B00003D0022C0DD008208AE6124B124A13495F
:1056C00013481B881288098800880094FFF7E0FDC2
:1056D000F1E7FFF78DFDEEE7CE64FF1FF564FF1FD6
:1056E000CA42FF1FA864FF1FF664FF1F9064FF1FDC
:1056F000AA64FF1FCB42FF1FA964FF1FC842FF1F00
:105700009464FF1FC042FF1FC242FF1FC442FF1F1D
:10571000C642FF1F10B502A804880B20002C10D130
:10572000496808784978090201430C48814209D147
:10573000022119800A4B59881170DB7800205BB276
:10574000537010BD074C0A20A142FAD102211980E2
:10575000034B998811705B79F0E7C0466E2A000010
:105760009462FF1F6F2A0000F7B5150008AA16887B
:105770004A680F4F14785278120222430A24BA4220
:1057800014D10122DBB2019200962A0005F0E0FE5E
:10579000041E0BD1074B1B68002B07D068782A78B2
:1057A0000002104342425041013098472000FEBDA4
:1057B000022900000865FF1F30B5012503790400A8
:1057C000BFB02B4225D01449408805F02DFA28425D
:1057D0000CD0124B01A95B8D00220B8002234B8061
:1057E0000F4B5B888B80608802F010FB0D4960884E
:1057F00005F01AFAC0070CD50B4B01A91B88002233
:105800000B8002234B80064B9B888B80608802F0C4
:10581000FDFA3FB030BDC0460065FF1FF442FF1FD8
:105820009462FF1FF864FF1F4E43FF1F10B5074C23
:105830000749200005F0AEF92000064905F0AAF955
:105840000721054A054805F067F910BDFFFF000074
:105850000065FF1FF864FF1FACBD0011F442FF1F7D
:1058600010B5024803F054F910BDC046B9570011F5
:10587000082110B50E240A4AC307DB170B405179E3
:10588000A1430B4353710223184202D051790B43B9
:1058900053710423184202D051790B43537110BD48
:1058A0006543FF1F0A2110B50F240A4AC307DB17FF
:1058B0000B401178A1430B431370830703D50623D4
:1058C00011780B431370400703D5012311780B4364
:1058D000137010BD6543FF1F10B5054B10241978D8
:1058E0000A00A243002801D022000A431A7010BD0A
:1058F0006543FF1F662110B52024134BDA788A43D5
:105900001979DA70A14324190C431C71542812D957
:1059100060200143197104210A43DA700222D97808
:105920000A43DA702022D9780A43DA704022D97803
:105930000A43DA7007E04428EDD83428EED824284A
:10594000F0D81428F2D810BD6543FF1FF8B50E2318
:10595000384C0500627926791A4011339E43364B44
:1059600062712671984204DD6E23E3716C3BA37172
:10597000F8BD324B984203DA1A23E3711C33F6E781
:1059800000232F49A371E37183B259182D4889B2BE
:10599000814224D9681D0A2100B205F0F9FF2A4B83
:1059A00000B29D4244DC05006421280005F0F0FFB0
:1059B0000A2100B205F0F4FF244F09B2E2797B5CC2
:1059C0001343E3710A21280005F0E2FF0A2100B227
:1059D00005F0E6FF1D4F09B27B5CA2790EE00121C4
:1059E0000A436271002D1CDA5B421DB20423A371CD
:1059F000A379632DD8DCFA22092DE3DC1343A371CC
:105A00000A21280005F0CCFF0F22114F09B27B5C60
:105A10001A4016431F229343627926711343637120
:105A2000A6E7FA239B009D42E2DB0123E371BBE77B
:105A30000500FAE76543FF1F1B4E00001DFCFFFF3A
:105A4000CB070000960F00000A270000F6BD0011EA
:105A5000E6BD001170B51B4D04002B7900290DD057
:105A6000802213432B71632C0BDD76236A7813435A
:105A70006B704023AA781343AB7070BD7F22134034
:105A8000F0E72300093306DA58236A7813436B7072
:105A9000AA786C23EFE70C4E002C0ADA202364422C
:105AA00024B26B700A21200005F07AFF09B2735C02
:105AB000E2E7092CF6DD0A21200005F069FF00B2BB
:105AC000335CEEE76543FF1FD6BD0011F8B50A4F02
:105AD00005003B780E00002B0CD0084C2000FEF790
:105AE00003FC33002A0020003978FEF7F1FC200087
:105AF000FEF738FCF8BDC0461565FF1F7043FF1F59
:105B000070B50A4E0A4D08223100280005F090FEBB
:105B1000002809D0074C31000822280005F060FE5B
:105B200009212000FFF7D2FF70BDC0466543FF1F6B
:105B30000D65FF1F0C65FF1F102110B50C4B3620A3
:105B40001A7898710A401A70DA7856310A40DA7079
:105B50006022197998701140223ADA71A2325A7192
:105B6000DF3A0A431A7106225A70FFF7C9FF10BDC7
:105B70006543FF1F10B5002824D0134C0A210223CF
:105B8000E05E05F005FF00B2FFF7E0FE0423E05EF3
:105B9000642105F0FDFE012100B2FFF75BFF207AD2
:105BA000FFF7A8FE0320FFF763FE0020FFF77AFE51
:105BB000064B1878053843425841C0B2FFF78CFEB7
:105BC000FFF79EFF10BDC0469462FF1FF564FF1FE4
:105BD00070B500250A4C2000A571FEF785FB102347
:105BE0003E212000074AFEF773FCA84200D13E3553
:105BF000054B20001D70FEF7B5FB0123A37170BD9E
:105C00007043FF1FC6BD00111565FF1F0200F0B5F0
:105C100001270A480A4E51188B1A002B00DCF0BDF0
:105C2000082415784308684038404000805B013CF8
:105C300058406D08002CF5D10132EDE7FFFF000060
:105C400006BE0011F0B500250F269D4200DBF0BD19
:105C50004C5D070944403440A400A0580135784009
:105C6000F3E70000F0B589B06A460D000B000F277E
:105C7000110010351C780133260024093E401670AF
:105C800054700232AB42F5D12023024AFFF7DAFF0B
:105C900009B0F0BD0CBE0011F0B54E780B7889B09C
:105CA00036020C00170001901E43012A61D9954B62
:105CB0009E4200D877E001339E421CD1062A17D1BC
:105CC000CA788B7812021A430B791B0413434A7962
:105CD00012061A438C4B5A6100221A705A808B4A62
:105CE0005A608B4A9A608B4ADA60002009B0F0BD96
:105CF00088225205EEE7884B9E423CD182498B7840
:105D0000002B00D0F6E00C2A31D10F22A378934368
:105D1000E2781202134322791204134362791206C5
:105D200013434B60E279A07912020243207A000407
:105D30001043627A12060243CA60E27AA07A120223
:105D4000024376484A81834208D804236E491422CC
:105D500001980B7005F044FD1420C7E71201D2181A
:105D600089235B059A42F0D801238B70BDE7022A94
:105D7000FAD00523EAE76A4A01239642E6D1FFF703
:105D800037FA052F0CD9E378A2781B021343227946
:105D900012041A4363791B061343624A0393136088
:105DA00005F0BEFCA1E7584D2B78002B9DD1AB78B8
:105DB000002B00D1A0E02B8901339BB20093B342AA
:105DC00000D091E0132AD4D9CF7C8B7C3F021221E2
:105DD00020001F43FFF71AFF874200D08EE0002EFD
:105DE0003DD1E378A2781B0213432279E9681204BB
:105DF0001A4363791B06134303930A228B4212D181
:105E0000FF23A370E370237163716B89002B09D1A9
:105E1000E37B227C1B0212041343A27B13431B0966
:105E200001336B8100226B89002B8ED0002A67D151
:105E3000686837013818000B6B69000303909842BB
:105E400005D9686105F064FDEB780133EB70686893
:105E50001022A11C381805F04BFD2E8145E76F89F3
:105E6000009A7B1E9BB293423AD1E278A378120249
:105E70001A43237905A81B04134362796C68120640
:105E80001A43EB6800920392211D0C22049305F043
:105E9000A7FC0120260004A940421036FFF7E2FECD
:105EA000013F012F17D1009A0B232861824200D0B5
:105EB0004CE704221C49200005F01AFD042203A926
:105EC000686805F04DFDE968039AFF23914200D10F
:105ED0003CE7F73B3AE73100FFF7C4FE1036DFE757
:105EE0000923B742A4D831E7009BB34200D9FCE6AE
:105EF00007232BE7022329E7032327E7062325E7C8
:105F00000A2323E7FFFE00007843FF1F0000011172
:105F1000FFFF00005048593601FF0000FFFF00114D
:105F200002FF000034F000408443FF1F10B5034C13
:105F30000B000122210000F06BFA10BDED60001192
:105F40000B8870B506000D000224162B11D92B000A
:105F50000322094900F05CFA041E0AD1074B2A8883
:105F60001B88191C934200D9111C300089B200F023
:105F7000EFFA200070BDC046196100113A65FF1F9D
:105F800010B54A780400013A0B000220012A07D814
:105F90000A78002A04D005222000024900F038FACD
:105FA00010BDC046476100110A7810B50B0004000F
:105FB0000220002A04D007222000024900F028FA1B
:105FC00010BDC046F36100110A7810B50B00040043
:105FD0000220002A04D009222000024900F018FA09
:105FE00010BDC0465962001110B5034C0B000B22C6
:105FF000210000F00DFA10BD8962001110B5034CAC
:106000000B000D22210000F003FA10BDFB6200110D
:1060100010B5034C0B000F22210000F0F9F910BD60
:10602000556300110A7810B50B0004000220002A05
:1060300004D011222000024900F0EAF910BDC04648
:1060400065630011002310B51322190000F0E0F978
:1060500010BD000010B5034C0B001722210000F00A
:10606000D7F910BDB7630011002310B5192219002C
:1060700000F0CEF910BD000010B5034C0B001B2240
:10608000210000F0C5F910BDF1630011F7B5848956
:106090000D0006000121002C22D000238268D35677
:1060A0001778002B1EDA0C2C1AD90C3CA4B2131949
:1060B00040880093230002F086FE431E9841013081
:1060C0007B06DB0F6B703F23013C1F40A4B228709E
:1060D000AF70AC80002C07D0B3680133AB600021F7
:1060E0000800FEBD0020EBE7AC60F8E70B7803701A
:1060F0004B8843704B881B0A83700B79C370042054
:1061000070470420022B06D10020537811781B021F
:10611000009A0B43138070470B8803700B881B0A8F
:106120004370022070470420009983420AD15378BB
:1061300010781B0203430B80D37890781B02034333
:1061400000204B807047F8B50D004B7801240021EA
:10615000461C03702B788B4201D82000F8BD6B7869
:10616000B01C4F1C012B10D1890069184B880222EA
:1061700033704B88B9001B0A7370691805F048FC2E
:1061800004360434A4B2F9B2E4E7122359436B187D
:106190005A88043132705B8810221B0A73706918A8
:1061A00005F036FC12361234ECE770B5049D14008D
:1061B0001E00052B01D8042070BD637812781B02E5
:1061C00013432B80E378A2781B02134302226B80D7
:1061D0002A71211D681D063E05F01AFCB2B22A8103
:1061E000E92AE8D82800A11D0A3005F011FC00209A
:1061F000E2E7002310B50A789A4201D8900010BD5A
:106200009A008A185488013304705488DBB2240A37
:106210004470948884709288120AC2700430EAE74D
:1062200010B51100029C062B04D004201022142B60
:1062300001D010BD022222714B7808781B02034363
:106240002380CB7888781B02034363800431601D70
:1062500005F0DEFB0020ECE710B50C788B780431FC
:106260005C43E4B203702200013005F0D1FB601CF6
:1062700010BD0420022B06D10020537811781B0298
:10628000009A0B431380704710B50C000A88023146
:1062900005F0BEFB208810BD70B504000D00049809
:1062A0001100012B01D8042070BD1678527812021B
:1062B000324302800200F13255701470E125002C47
:1062C00000D10C35023B9AB24280AA42EBD802318F
:1062D000043005F09DFB0020E6E70420009983428E
:1062E0000AD1537810781B0203430B80D37890783F
:1062F0001B02034300204B80704710B50C000A8836
:10630000023105F085FB208810BD000070B5012129
:106310001E000420049C0E400B4218D1CB40DDB27D
:106320008D4214D90A49DBB2098899420FD3230060
:10633000EE331D703300580011184978165C0902BD
:10634000314301332152D9B28D42F4D8002070BDBF
:106350009043FF1F10B50C000A88023105F058FB6E
:10636000208810BD10B50C788B7804315C43E4B202
:1063700003702200013005F04BFB601C10BD10B50E
:1063800011000298032B01D8042010BD1478527814
:10639000043B120222430280CA788C781202224304
:1063A00042809AB28280EB2AEED80431063005F0A2
:1063B0002FFB0020E9E710B50C000B8803700B8859
:1063C0001B0A43704B8883704B881B0AC3708A88F2
:1063D0000430063105F01CFBA088043080B210BDEB
:1063E0000420012B03D100201378009A137070470A
:1063F00010B50C000B8803700B881B0A43704A8889
:106400000230043105F004FB6088023080B210BD18
:10641000F0B589B003931E4B029242000700D05A98
:10642000019102F020F81325061E2DD0029B0124B5
:106430000370019B002B04D00019039998470019A1
:1064400084B26B461B7A5BB2002B0FDA1021380046
:1064500002F01CFB1925002813D130003219E1B2DB
:1064600002F066FC051E0CD10C34A4B2042304AA6D
:10647000380005A993800696948101F0AFFD051EB2
:1064800002D0300005F064F9280009B0F0BDC04624
:106490003865FF1F70B505000C0000280CD00020E7
:1064A000814209D010222000044905F0B1FA0120F0
:1064B0002B7823736B78637370BDC0464CBE00119C
:1064C000F0B506000D0017001C0085B002291BD096
:1064D0000020102907D1022B07D0102B03D115E083
:1064E0000020102C08D005B0F0BD69463800FFF739
:1064F000D1FF2A0069460BE069463000FFF7CAFF6A
:1065000022006946380004E0022BE9D12A00390054
:10651000300005F015FBE6E7031CF02800D9F02356
:10652000032008499AB2013A0B80D3170340064969
:106530009B189B100B80D30F04499B185B100B809A
:106540007047C0469443FF1F9243FF1F9043FF1FB5
:10655000034B1B888B4202D3024B4000C152704751
:106560009443FF1F3865FF1F014B4000185A7047C6
:106570003865FF1F1722014B1A8070473865FF1FCF
:1065800070B505000E2005F003F9041E13D0D023CA
:10659000037000230622837007494570033005F01D
:1065A00037FA064B2100DA8A62811B7E2373044B83
:1065B000187805F005FA70BD5465FF1F4465FF1F8C
:1065C000E443FF1F262803D8024B4000C05A7047FF
:1065D0000148FCE79643FF1FFFFF000070B506006F
:1065E0000C00094D1C220021280005F001FA074B80
:1065F0001E70074B1C7005F00BF90123002801D019
:10660000002312202B7070BD4465FF1FE443FF1F61
:106610006565FF1F70B505000D4C0800E260A160C4
:1066200010220021656005F023FB012803D1102111
:10663000A06802F058FD10220021280005F018FB88
:10664000012803D11021606802F04DFD70BDC046E5
:106650004465FF1F70B5041E05D1002903D0062232
:106660000D4805F0D5F90D4B1D78012D11D1002CE9
:1066700005D102221A7005F0EBF8280070BD002247
:106680001A70074B1B78FF2BF7D02000FFF778FF1D
:10669000F3E70025F1E7C0465465FF1F4465FF1F7F
:1066A000E443FF1F030010B5002801D1002010BDF6
:1066B00000780B4A002803D15988D1821B791376C0
:1066C0001378022BF2D10023984200D103331370C8
:1066D000044B1B78FF2B01D0FFF752FF0120E6E7A8
:1066E0004465FF1FE443FF1F002911D000280CD090
:1066F0004B79012803D140225242134303E03F2249
:106700001340032802D001204B7170474022F4E768
:106710000800FAE770B5094D0100287800280BD071
:10672000074C0622200005F073F921002878FFF7B6
:10673000DBFF200005F04CFA70BDC0466465FF1F0A
:106740003E65FF1F00290AD0012808D13F224B795E
:106750009343C02B03D0403B5A425341981C70478F
:1067600070B5174D06002B78FF2B15D00A2005F0C9
:106770000FF8041E10D0D0230370C83B8370114B58
:1067800011491B784670C3700622043005F040F9A9
:106790002100287805F014F90C4B1B78012B0DD142
:1067A0000B4B1B68002B03D09B68002B00D0984735
:1067B000084B04211878084A05F0B2F970BDC046AC
:1067C000E443FF1F6465FF1F3E65FF1F6065FF1FF9
:1067D0008C65FF1F9065FF1F60EA0000014B986801
:1067E0007047C0464465FF1F014BDB68186870475F
:1067F0004465FF1F074B10B5DA6813680133136057
:10680000054B1878FF2803D08021C90105F040F915
:1068100010BDC0464465FF1FE443FF1FF7B50E00DF
:1068200002F0C8F8051E1CD00E4B06621F78002F20
:1068300000D10778AB791020019304F0A9FF041E62
:106840000FD0D0230380C73B8370019BE91DC37029
:106850000622043005F0DCF821003800E66005F07F
:10686000AFF8F7BDE243FF1F014B18787047C046F1
:106870006465FF1F054B002805D1054B1A78054BB1
:10688000002A00D1014B18007047C0465465FF1F15
:106890006465FF1F3E65FF1F014B58687047C04687
:1068A0004465FF1F024B1868431E9841C0B27047F1
:1068B0006865FF1F421E03000120152A03D9FF3B14
:1068C0005A425341D8B27047F0B51C0000230E0065
:1068D00085B0039002920B70029A934201D300207C
:1068E00019E0E55C5A1CD2B2002DF8D0029851197B
:1068F0008142F4DC0233DFB2A35C18000193FFF79E
:10690000D9FF002807D0013D019A0399EBB23370FB
:106910008A4202D1E01905B0F0BDDB19DBB2DBE73A
:1069200010B50C0002F09EF803001220002B03D0DB
:106930002100588804F0A4FE10BD000070B50E4D73
:1069400084006359002B15D0186A002801D004F088
:10695000BFFE2B59586A002801D004F0B9FE2B590C
:10696000986A002801D004F0B3FE285904F0B0FE64
:1069700000232B5170BDC0467465FF1F1C4B70B5C2
:1069800004000E00150099420AD11A4B1B68002B17
:1069900001D1122070BD1B68002BFAD09847F9E78F
:1069A000154B994215D1134B1B68002B0AD01B685D
:1069B000002B07D09847002804D1104B1C70104BB7
:1069C0001D70E7E729002000FFF7AAFF0028E1D1AA
:1069D000F3E7080001F0EEFF0028DAD00378032087
:1069E000A342D7D12900300004F04AFED2E7C046C6
:1069F000FEFF00007065FF1FFFFF00006D65FF1FB9
:106A00006C65FF1FF7B50400808801F0D3FF0025F7
:106A1000A84203D00578A08802F008F81C4E33780D
:106A2000002B1FD0AB421DD11A4B28001978FFF75D
:106A300077FF002818D000233370A3790820A778A7
:106A4000A688019304F0A4FE011E0DD0D02303708C
:106A5000CA3B8370019B477086808371280004F0D5
:106A6000AFFF01E0002DE8D1A0880B4B8200D35886
:106A7000002B01D0FFF762FF1721A088FFF768FD08
:106A8000A08801F027FDA08801F0FEFDF7BDC046FB
:106A90006D65FF1F6C65FF1F7465FF1FF0B587B044
:106AA0001D000CAB1B88070001930DAB1B88142045
:106AB00002930EAB1B88160003930FAB1B8800914B
:106AC000049310AB1B88059304F062FE041E1AD0D9
:106AD000D0230370CB3B47708370C6700622290019
:106AE0000430002D11D004F093FF019B210063813D
:106AF000029B0098A381039BE381049B2382059B57
:106B0000A37404F05DFF07B0F0BD04F071FFECE783
:106B1000F7B5009308AB1B8807000C200D0016008A
:106B2000019304F035FE041E13D0280001F042FF4B
:106B300000280FD00078D0232370C93BA370009B9E
:106B400021002381019B6770A580E680638104F0AA
:106B500037FFF7BD014B1878EDE7C046E443FF1F50
:106B600013B5040064890389C2888188C0780094C1
:106B7000FFF7CEFF13BD000010B5044C20680028BD
:106B800003D004F0A5FD0023236010BD7865FF1F2E
:106B9000A122F0B5818892004A43384B384F1B68D8
:106BA00004009B189D2292009B18827989B01A607C
:106BB0003B68002B5FD01D78324B1B68002B04D044
:106BC0005B68002B01D00020984726000836310072
:106BD000E079FFF7B7FD237DE0710200E0780493D0
:106BE000638A29000393238A0293E3890193A3888C
:106BF00000933300FFF752FFE378002B0BD1E289BB
:106C0000A379A18802920196E279280000920122DC
:106C100001F0DAFEE0703B68002B20D0FFF7ACFFFC
:106C2000194D287800281AD0184B1978FFF778FEEC
:106C3000002814D02B78E67808200793A78804F062
:106C4000A7FD011E09D0D0230370CA3B4670837094
:106C500087808671079804F0B3FE00232B701721FC
:106C6000A088FFF775FCA08801F034FCA08801F033
:106C70000BFD09B0F0BD064B9DE7C0463409FF1F70
:106C80007865FF1F8C65FF1F6D65FF1F6C65FF1F1B
:106C9000E443FF1FF8B5070008000E0001F08AFE6C
:106CA000041E18D02620FFF78DFC051E00D1257884
:106CB000062004F06DFD041E0DD00021062204F014
:106CC00097FED0232370C23B21006770A370A6807B
:106CD000E8B204F075FEF8BDF0B585B001930AABDB
:106CE0001B78070002930BAB1B7808000D00009285
:106CF000039301F05FFE061E22D0102004F048FD31
:106D0000041E1DD01022002104F072FE2620FFF781
:106D100059FC002800D13078D0232370C13BA370E8
:106D2000009B21002372019B67706372029BA58008
:106D3000A372039BC0B2E3720C9BE36004F040FEBD
:106D400005B0F0BDF7B50D00019001F033FE071E50
:106D500020D00E2004F01CFD041E1BD02620FFF7BF
:106D600031FC061E00D13E78D0232380C53B06228D
:106D7000A370F91DE01C04F04BFE019B2A00638107
:106D80000123DD401A401D40210022736573F0B2DB
:106D900004F016FEF7BD0000F0B585B002901000BB
:106DA0000D0017000A9E039301F004FE041E31D06B
:106DB000029B002B2ED1039B02795B0724D5122363
:106DC00013430422002E08D10B99002905D10C99F8
:106DD000002902D10D9900291AD01A430D9B227166
:106DE000002B00D0C9E0002E00D1CFE0002D00D054
:106DF000CCE0606A002801D004F06AFC1C2130005D
:106E000004F056FD606205E002239A430E33D7E793
:106E100093432371654BBA00D458002C00D1AAE0EB
:106E2000002E10D0236A002B03D11C2004F058FC44
:106E300020625E4BBA00D358186A002803D01C2287
:106E4000310004F0E5FD0C9B002B12D0574CBB0029
:106E50001D596B6A002B03D1162004F041FC6862B7
:106E6000BB00E358586A002803D016220C9904F09E
:106E7000CFFD0D9B002B11D04C4DBC006659B36A61
:106E8000002B03D1142004F02BFCB0622B59986A1C
:106E9000002803D014220D9904F0BAFD380001F047
:106EA00089FD051E67D0414BBA00D358002B62D034
:106EB0001A6A3420002A00D11C389A6A002A01D0AC
:106EC000143080B20B9A002A01D01C3080B25B6A69
:106ED000002B01D0163080B204F05AFC041E4AD0B8
:106EE0001822002104F084FD2620FFF76BFB01909F
:106EF000002801D12B780193D0232370029B20001E
:106F000063700A23294EA370039BBD00A371AB5984
:106F1000A780196A1830002905D01C22A06004F04F
:106F200077FD200034307359996A002907D0030097
:106F300014221433E060029304F06AFD02980B9B64
:106F4000002B08D003001C221C330B9920610293F4
:106F500004F05EFD02987359596A002903D0162285
:106F6000606104F055FD6B462100187904F028FD9E
:106F70003800FFF7E3FC05B0F0BD10220D9B0D9922
:106F80001B69A018236204F043FD2CE70B9B002B28
:106F900000D13FE7012D00D03CE7606A002801D016
:106FA00004F096FB1C210B982AE7C0467465FF1F6E
:106FB00010B5044C2068002803D004F089FB00239E
:106FC000236010BD6865FF1F0B4B07B51A68002AC8
:106FD00001D100200EBD6946531C012012780731F3
:106FE000FFF772FC0028F4D002780123100018404B
:106FF0001A42EED0EEE7C0468465FF1FF0B51F4F82
:1070000001203B6887B0002B25D09B78059300F0CA
:10701000B3FB002821D00A20FFF7D4FA04000B208C
:10702000FFF7D0FA164B05001E78731E9E413B6891
:10703000F6B2191DD878FFF757FB3B682900DA7ABA
:10704000043303929A790193029200903300200056
:10705000059A04F0B5FD07B0F0BDFFF7B5FF0028B5
:1070600005D00620FFF7AEFA04000720D8E7082075
:10707000FFF7A8FA04000920D2E7C0466865FF1FA1
:107080006465FF1F70B50A4E040033780D00FF2BB6
:107090000DD0042004F07CFB011E08D0D023037027
:1070A000CE3B45708370C470307804F089FC70BDAD
:1070B000F443FF1F70B5040006200D0004F068FBC8
:1070C000011E0AD0D0230370CD3B8370054B447062
:1070D0001B688580187804F073FC002C01D0FFF742
:1070E00067FF70BD6865FF1FF8B5264F06003B6857
:1070F0000D001124002B05D10522234B1B781342D0
:1071000002D112242000F8BD204A10241268002A5F
:10711000F8D01278002AF5D0DB0719D52B789A1E03
:10712000012A1AD80C2004F0DBFA13243860002856
:10713000E8D000230A22437029000670023004F0D0
:1071400067FCFFF75BFF041E0AD0FFF731FFD9E7AA
:1071500000F012FB0028E1D1E4E7002BE2D0D0E7F9
:107160000B4B1B78032BCDD11D20FFF72BFA094BBE
:1071700018800028C6D0084B04211878074A04F06C
:10718000CFFCBFE76865FF1F6565FF1F8465FF1FB4
:107190006465FF1F6265FF1F9065FF1F60EA0000C6
:1071A000F7B50193194B14001A78052306000F0058
:1071B00012201A4221D0012920D1154B1D68002D23
:1071C0001BD002201F2C18D8002C02D0019B002BB2
:1071D00013D0104B1F221E706E1C0021300004F0D3
:1071E00007FC01992200300004F012FC310020005D
:1071F0002C70002F06D004F09BFBFEBD064B122026
:107200001D68DCE704F014FAF7E7C0466565FF1F68
:107210008465FF1FF443FF1F8065FF1FF8B50F4E05
:1072200012243368002B17D01B780F3C834213D1F4
:1072300000250B4F0221387804F022FB094B042172
:1072400038781D8004F01CFB074B28001D80336834
:107250005C7004F0EDFB04002000F8BD6865FF1FC2
:107260009065FF1F7C65FF1F6265FF1F70B50128D9
:1072700023D11B4C2388002B03D01A4A1578002DEC
:1072800007D0194B1B68002B02D01878FFF7C6FFF8
:1072900070BD3B2B02D93C3B2380F9E7134E022102
:1072A000307804F0EDFAFA222388920002215A4342
:1072B000307804F03DFA2580EAE70B4B1B68002B81
:1072C000E6D00B4B1B785B07E2D5084B0221187800
:1072D00004F0D6FA0022024B1A80FFF769FED7E7C6
:1072E0007C65FF1F6065FF1F6865FF1F9065FF1FBE
:1072F0006565FF1FF8B51E4D2868002803D004F00F
:10730000E7F900232B601B4E3068002803D004F0FF
:10731000DFF900233360184F05243B781800204024
:10732000234221D0154800F02BFA3B78234213D09A
:10733000202004F0D5F92860002813D02022002155
:1073400004F056FB202004F0CBF9041E306005D079
:107350002022002104F04CFB002004E0286804F007
:10736000B7F92C601320F8BD00F00AFAF4E7C04624
:107370008465FF1F8065FF1F6565FF1FE843FF1FD2
:1073800010B50A4C23681A1E0ED0002808D101300F
:10739000587004F04DFB002805D02368002B02D064
:1073A0000021FFF787FE0122100010BD6865FF1F56
:1073B000F7B5274E050033680191181E21D05C787F
:1073C000244F012C30D1FFF7FFFD002825D02000ED
:1073D000FFF7F8F80400412814D91F4B0221187850
:1073E0001E4A04F09DFB1E4B3C3C1C80022233686D
:1073F0005A703B78002B14D128000199FFF75AFEF0
:107400000120FEBDFA2292004243002AEED0124B28
:107410000221187804F08CF9E8E7FFF7D3F80200AE
:10742000F3E700233B70EBE73B78002BE8D1032028
:1074300004F0AEF9011E08D0D0230370CC3B457098
:1074400083703368187804F0BBFAFFF7B1FDD7E713
:107450006865FF1F6065FF1F9065FF1F60EA000001
:107460007C65FF1F10B51749838802008B4220D02E
:1074700011D815498B4217D0144900205B1899B2D6
:10748000012907D8926811785A425341D8B2FFF7C0
:10749000F9FD012010BD0E4A00209B1807229BB267
:1074A0009A424041C0B2F5E783681878FFF768FF59
:1074B000F0E7836899785A78090218781143FFF742
:1074C00077FFE7E70A20000006200000F8DFFFFF53
:1074D000AFDFFFFF014B18707047C046F543FF1F39
:1074E00010B5064C207001F041FA207804F070FAD3
:1074F0000521207800F062FD10BDC0469065FF1F99
:107500000BB273B50D00002B00DBC4E0884B18787C
:1075100004F086F9041E0ED00378912B0FD0A22B15
:1075200000D1A1E0834B1878FF2852D0210004F04D
:1075300047FA00284DD180200002684076BD43788C
:107540000F2B76D013D8052B70D00E2BEAD1808864
:10755000794B98422BD8794B98421BD8784B98425C
:10756000E0D1A3681878591CFFF774F838E03E2B77
:10757000D8D18378032B74D06CD8012B6ED0022B1A
:10758000D0D1704B1B68002B23D05B68002B20D020
:1075900098471EE06C4BC0180C28C3D804F0A0FA22
:1075A0001DC2C2150BC20B0B0B3223C23C00674B32
:1075B000C0180728B6D8664B1B68002B09D01B687B
:1075C000002B06D0200098470AE0A3681878FFF740
:1075D000C7F8200004F064F8ADE7A068FFF762F890
:1075E00000289FD0F5E7A3681B78002BF1D0554BFE
:1075F0001B68002BEDD01B68002BEAD021005548FA
:107600009847EDE74F4B1B68002BE2D01B68002B1F
:10761000DFD021005048F3E7504B1B68002BD8D037
:107620005B68002BD5D021004348E9E7FFF7EAF972
:10763000CFE780884A4B984203D04A4B984200D00B
:1076400070E7464B1B68002BC3D05B68002BC0D093
:107650002100D5E7153B012BBBD963E7FFF798FA6B
:10766000B7E7FFF77DFAB4E73F4B1B78042B07D150
:1076700000236A4613800179408800F0C5FCA8E722
:10768000364B1B68002BA4D05B68002BA1D00100F7
:10769000364898479DE7012421420AD0294B1B68B0
:1076A000002B04D05B68002B01D0002098470120FC
:1076B00043E78B070AD5264B1B68002B04D05B6879
:1076C000002B01D020009847022036E70421280033
:1076D00008400D4200D131E7254E3388002B21D0E0
:1076E000013B9BB23380002B1AD1FFF7DBF8002857
:1076F0000AD0204B1C70164B1B68002B04D05B6813
:10770000002B01D020009847FFF7C6F8694601F02A
:1077100001FD6846FEF7FEFF1D20FEF753FF308097
:1077200004200AE7024B187804F0AAF8F8E7C046EC
:107730009065FF1FF543FF1F0E2000000120000091
:10774000091000008865FF1FFEDFFFFFAFDFFFFFAE
:107750008C65FF1F0C2000000B2000007065FF1FD0
:107760000D200000132000006565FF1FFFFF0000D3
:107770006265FF1F6065FF1F10B501F09BF910BD2A
:10778000014B18607047C0468C65FF1F0B880020B6
:10779000162B01D817230420014A13807047C046D6
:1077A0003A65FF1F00207047074A03001188814295
:1077B00007D091880020994202D101308000101832
:1077C00070470020FAE7C0469865FF1FF0B58F7834
:1077D00006000D00C5B01E2F15D1FFF7E5FF051EF1
:1077E00003D10024200045B0F0BD00223B00310051
:1077F000C078009200F0B2FB0400A81C00F0D2FB9D
:10780000FF23EB70EEE7264B062403931B78FF2B38
:10781000E8D0182FE6D87B08224A013BDB00029211
:107820009A589446002ADDD0029AD3185B68002B40
:10783000D8D00878002802D14B78012B02D1062439
:10784000122FCFD107AFAB88697800976446AA683A
:10785000A047041EC6D1AB78029A5B08013BDB004F
:10786000D318390030005B689847041E0BD1AB7801
:10787000042BB6D0039A310010782200009700F054
:107880006DFB0400AEE76A78002AABD1AA7805A99F
:107890003B88087130000A704B80FEF747FBA0E779
:1078A000F843FF1F5CBE00111D4B37B50500984221
:1078B0000BD000290AD1FFF777FF002805D119481E
:1078C000FFF772FF002800D0058037BD01291AD1CB
:1078D000FFF76AFF041EF8D001235B420380A37800
:1078E000FF2BF2D0FE2B07D00023E0781422009368
:1078F00029001E3300F032FBA01C00F053FB0123D3
:107900005B426380E1E70229DFD1013901F0BEF873
:107910000028DAD12800FFF747FF041EDFD1D4E7A3
:10792000FEFF0000FFFF0000022210B5074B52428D
:107930001A80074801325A809A80DA8000F07EFA75
:10794000044801F025F8002010BDC0469865FF1FCF
:10795000CD770011A97800110388F7B50400002B3A
:1079600002D102252800FEBD426802211378254875
:107970005268FEF7A5FD00282ED0234F01253A8836
:10798000002AEFD0802321885B0201259B1A9942AF
:10799000E8DC0C2003F0A4FE061E31D03B882288D0
:1079A0009C4600231800019561469DB2491989B291
:1079B000AA421BD8002801D062443A80002330003C
:1079C000082208C0210004F023F8104A1368002B95
:1079D00013D100251660C5E76268022113780C48B0
:1079E0005268FEF76DFD0028C7D1BAE760681D0137
:1079F0004019418101330198D6E71A001B68E6E778
:107A00001325AFE7CABE0011F643FF1F9465FF1FA1
:107A1000C8BE0011014B18707047C046F843FF1FE5
:107A200014230A0010B51A40194204D00122102173
:107A300001F048F810BD4B06F9D4012088434000FE
:107A4000F8E710B514008B0604D50122102101F0CF
:107A500039F810BD08230A001A40194202D14BB26E
:107A6000002B0FDA102101F02DF8002808D0230098
:107A7000F2331B78002BECD0F1342378012BE8D1C2
:107A80000020E6E703208907FAD4E2E7F0B51F00FB
:107A9000184B85B01C68019002910392002C27D1ED
:107AA000200005B0F0BDA5683301ED186B89019A7F
:107AB000934211D3029A93420ED8002F04D10A9B0D
:107AC000002B10D12C00EBE73B002978039A686863
:107AD000FEF7F6FC0028F2D10136B6B2A388B34215
:107AE000E1D82468DAE7A3680A9A5B891380E9E79A
:107AF0000026F3E79465FF1F37B50C000A88498814
:107B00000123914217D3002A15D0651D23792A003D
:107B100002210A48FEF7D4FC102300280BD0237959
:107B20006188208800242A000094FFF7AFFF0A2311
:107B3000A04200D0230018003EBDC046CABE0011BE
:107B400013B50A0008884988012388420BD8002809
:107B500009D00024137905320094FFF797FF0A2318
:107B6000A04200D02300180016BD13B50A000888F3
:107B70004988012388420BD8002809D000241379B2
:107B800005320094FFF782FF0A23A04200D02300B1
:107B9000180016BDF0B58BB003904A8808880E0017
:107BA0000123824255D3002853D00023012704AC7F
:107BB00023700022718813000092FFF767FF051EF3
:107BC0003ED02078002835D12B78022B18D1677051
:107BD0006A8983000130E31880005A8069680222B4
:107BE000201803F015FF23780133DBB22370042B38
:107BF00019D93B006889013080B2002BD9D01FE031
:107C000002236370122358436A89231804305A8070
:107C100069681022201803F0FBFE23780133DBB2E1
:107C20002370002BE5D10C4A6B899B185A425341B3
:107C3000DBB2DFE76378012BE4D12B78022BC7D0CE
:107C400022780A23002A04D021000398FEF798F92D
:107C5000002318000BB0F0BD0100FFFF0F4BF0B583
:107C600004001868002816D083685D89A54207D8EB
:107C70008288AE18B44203DA12019A18934201D1F5
:107C80000068EFE71E005F891036A74204D1002983
:107C900000D00D801800F0BD3300EFE79465FF1FA2
:107CA00070B505000C0008880021FFF7D7FF03001E
:107CB0000120002B04D022002800197AFFF7C1FE12
:107CC00070BDF7B50C00002501902300EE331B7842
:107CD000AB4201D800200AE06B00E65A00213000D8
:107CE000E718FFF7BBFF002802D126800130FEBD58
:107CF000017A0198FFF794FE002802D03B88238088
:107D0000F5E70135EDB2E0E710B504000888002181
:107D1000FFF7A4FF03000120002B03D02000197AF5
:107D2000FFF77EFE10BD0000054B1B68002B01D144
:107D3000180004E09A6852898242F6D19888704708
:107D40009465FF1FF0B50E27002687B0039302ABA2
:107D5000FF183E8005001F4B40891400984207D051
:107D60002B78013000976A6880B2FFF78FFE06001B
:107D700002212B7818486A68FEF7A2FB00280FD072
:107D80006C892000FFF7D0FF002802D0013C0419C5
:107D9000A4B2039B002B00D01C80300007B0F0BDC4
:107DA00002212B780D486A68FEF78AFB0028E7D18C
:107DB00002212B780A486A68FEF782FB002807D068
:107DC000002EDED03B88A342DBD17489013CDFE783
:107DD0006C89DEE7FFFF0000CABE0011C8BE0011BB
:107DE000C6BE001110B50C00FFF7DEFC0300022038
:107DF000002B0AD0002C00D023609B781720FE2B8C
:107E000003D00138FF2B00D1002010BD73B50D0049
:107E100001A904001600FFF7E5FF172805D0002E82
:107E200004D129002000FEF727F976BD0122102198
:107E3000200000F047FE0028F3D0F6E7014B186061
:107E40007047C046A465FF1F37B56B469D1D0100F6
:107E500004000222280003F0C3FC2B88B02B0ED1B3
:107E60002379122B09D12300FA331B78012B06D179
:107E70000121608800F0E0F801E01B2BF8D037BD4D
:107E800010B5054B0421187000F098F8FFF74CFD71
:107E9000FEF770FB10BDC046A865FF1F0020F0B5BF
:107EA0000BB20F0087B0834234DA274B187803F007
:107EB000B7FC051E2BD00378A02B25D103AE3100D3
:107EC000FEF7E4F8041E0BD1B378DB0724D51F4B73
:107ED00006341B68002B03D03100688898470400E3
:107EE000A868002801D003F033FC002C08D1184A00
:107EF000039B1340174A934206D0B3781B2B03D041
:107F00000121688800F098F8280003F0C9FB802060
:107F10000002784007B0F0BD0F4B1B68002B10D05B
:107F2000310068889847041EDAD07378002BD7D1C7
:107F3000B27801A90A704B800C716888FDF7F6FFD2
:107F4000CEE70624F1E7C046A865FF1FA065FF1F26
:107F500000FFFF0000011200A465FF1FF7B50190AC
:107F6000FC200D0017001E0003F012FC040013207B
:107F7000002C12D0B02320002370089BF4226770DD
:107F8000658026710830002B08D0190003F040FDF1
:107F90002100019803F014FD0020FEBD089903F0B4
:107FA00027FDF5E710B5041E06D00078FD2803D89C
:107FB00003F076FCFF23237010BD00000A1F93B26C
:107FC00010B504000220032B05D882400020024B8C
:107FD000D1529B189C7010BDC865FF1F0B8870B5EF
:107FE000043B04000D000220032B0BD801212000CC
:107FF00000F04CFD03001420002B03D029002000CA
:1080000000F0DEFB70BD000007B51300034A0092CC
:108010000A00012100F02CFC0EBDC0464582001173
:1080200007B5019203220092024B0A00122100F0D0
:1080300049FC0EBDC382001107B56B4601AA118031
:108040000449D88008780633012802D1190003F0CA
:1080500077FC07BDA965FF1F0C4B10B518700023F6
:10806000FF210B4A1380138193819380094A538027
:108070001370517293819372D174D38213755177B7
:1080800003F086FD00F0FCF910BDC046D865FF1F67
:10809000C865FF1FAA65FF1FF0B58DB06B460020B5
:1080A00003910C229B5E834200DBB0E05D4B1878AD
:1080B00003F0B6FB051E00D1A4E00378902B00D09E
:1080C0009DE006AF01004688380000F013FA796899
:1080D0000400002900D19CE03B88052B6ED13B8930
:1080E000032B1CD905AC200000F0A2F86288172AE7
:1080F00061D83989131D994231D1796823780431C7
:108100000291D90738D5607800F08EF9071E06D0A5
:10811000002303712378012B08D0132B23D0A868E8
:10812000002800D178E003F013FB75E06288029923
:1081300009A800F0A6F80290380000F08BF909AA0F
:108140002378387A0192002231000092029A00F0DE
:1081500012F9380000F064F9029B002BDFD03000E8
:1081600000F080F9DBE70378032BD8D1628802990D
:1081700009A800F0D6F8DEE7122B13D1029909A85E
:1081800000F0B5F8021EEAD127498B88002BC6D033
:10819000887909A92378019161780091310000F074
:1081A000EAF8BCE7002302AA93833000617809AAA9
:1081B000FFF72AFFB3E71D4B0993F6E7042B02D024
:1081C0009A1F012AABD8184A043B9B00995A0029F0
:1081D000A5D0D218907831003A0000F0AEF800280F
:1081E0009DD13B88042B03D001213000FFF724FFF1
:1081F000012C04D1A868002801D003F0A9FA2800B6
:1082000003F04EFA8020039B0002434018000DB09B
:10821000F0BD012800D182E701213000FFF70CFFFB
:10822000EDE7C046D865FF1FC865FF1F01001700B6
:108230000B7803704B784370CB788A781B0213431A
:10824000438070470A88030002700A88120A42704D
:108250000A88012A06D14A8882704A88120AC270A6
:108260000420704702208242FBD14A8804309A7071
:108270004A88120ADA708A881A718A88120A5A7130
:10828000EFE710B50400012082420CD94B780A7840
:108290001B0213432380834206D1CB788A781B02CA
:1082A00013436380002010BD022BFBD1CB788A786A
:1082B0001B02134363804B790A791B021343A3808B
:1082C000F0E70B8803700B881B0A43704B888370A0
:1082D0004B881B0AC3708B8803718B881B0A437100
:1082E000CB888371CB881B0AC371082070470300B9
:1082F0000120082A14D14A780878120202431A8011
:10830000CA788878120202435A804A7908791202A0
:1083100002439A80CA798879120202430020DA80E7
:10832000704710B504000120022A05D100204B78C7
:108330000A781B021343238010BDF8B506001020F5
:108340000F00150003F024FA04000120002C0ED0C9
:10835000A0230C22290023806780201D002D07D038
:1083600003F056FB2100300003F02AFB0020F8BD8B
:1083700003F03EFBF6E7F7B51E00009008AB1420B3
:1083800017001D78019103F003FA041E12D0A223F6
:108390000370019B47704380099B057146710C2255
:1083A0000830002B07D0190003F032FB21000098A1
:1083B00003F006FBF7BD099903F01AFBF6E737B5A2
:1083C000041E0FD04388002B0CD00025C188132336
:1083D000007A172201950095FFF7CDFFFF236580F6
:1083E0006372257037BD000010B50C4904004A883F
:1083F000002A09D08B89002B05D00020CB8A0222CD
:10840000834201D010BD012213000A204343002003
:108410004032C854C81842800472F3E7AA65FF1FAF
:108420000023438003707047094B00211A0010B5E8
:108430005C88002C06D01C79844203D10A234B436C
:10844000D01810BD01310A330329F1D10020F8E71B
:10845000AA65FF1F10B50400407A03F021FAFF233C
:10846000637210BD7047043010B580B203F040FB5A
:10847000002803D00421494203F0BAF910BD0000DE
:1084800070B50025104CA0682580A581A580A84264
:1084900002D003F05DF9A56000250C4C0C4B606D1B
:1084A0001D80230058331D70A84202D003F050F9FC
:1084B000656500256068002801D003F049F90135A1
:1084C00008340A2DF6D170BD7066FF1F1466FF1FB9
:1084D0006466FF1F70B5041E09D1054D2880A88170
:1084E000A880A868002802D003F032F9AC6070BD03
:1084F0007066FF1FF0B54B8885B001930023436081
:108500000A7905000F00022A00D07BE0CA88032AFE
:1085100017D98B685E7819783602DC78D8790E43E3
:1085200099781B7A24021B020C43034353495BBA1C
:108530000B80331D93421ED1042C04D0631F022BE9
:108540000ED9012015E0019A4D4B1201D35A002B90
:1085500006D00198FFF7BEFF4A4A13690133136141
:108560000421B8682E812C80494203F041F96860EB
:10857000002005B0F0BD434D042C06D0631F022B34
:108580000FD9EB680133EB60DBE7019A3C4B12013A
:10859000D35A002B05D00198FFF79CFF2B690133BC
:1085A0002B61374B30000293019B029A1B01019310
:1085B000002301998C468B52130063449C800393E3
:1085C0009E81FFF750FF039B041E986016D0042184
:1085D000B868494203F00CF9FA880100043A200017
:1085E00003F016FA0199029AFB888A5A043B9B18F9
:1085F000029A8B522B6801332B60A2E7AB690133DF
:10860000AB619EE71E4B0293019B1E01029BF35A36
:10861000002B2DD002998C19A068002828D0012A9F
:1086200026D1FA889B189BB27352A189994217D31D
:108630009B1AC018B96803F0EBF9029BA289F35AA0
:10864000934200D07DE700222B81A3882B80A36872
:108650006B60029BF2520B4A53680133536070E720
:10866000084A9368013393600198FFF733FF68E786
:10867000044A536901335361F6E7C046DA65FF1FC8
:108680007066FF1FE065FF1F70B5051E15D10B4C0E
:108690000B4B1880230058331870606D002802D0EF
:1086A00003F056F86565250050356068002801D054
:1086B00003F04EF80834AC42F7D170BD1466FF1FCA
:1086C0006466FF1FF0B51700A12285B092000193E8
:1086D0004243394B06001B680C009B18D933FF330B
:1086E0001D78FDF741FF0430854204DD3000FDF7C1
:1086F0003BFF0430C5B2BD4207D33A000021300031
:10870000019B03F03DF905B0F0BD2900380003F0EE
:108710004FF82300C6B250331E700393019B29000B
:108720006365380003F09CF8CBB20293002B02D0B3
:10873000039B01361E7000262300503303931B78E1
:10874000B34204D8606D002831D10020DBE7029AE3
:108750002800002A04D0013B1000B34200D02800BA
:10876000F700E719387003F063FA786000280ED03C
:108770003A78019903F04CF9019A3B780136D31805
:108780000E4A0193D369F6B20133D361D4E7039B58
:1087900018706065A74205D1084A1320D36A0133D7
:1087A000D362B0E7606802F0D3FF0834F2E702F06A
:1087B000CFFF00236365C8E73409FF1FE065FF1F93
:1087C000F7B50D0007000421686803F011F82B8944
:1087D000040003702B891B0A43702B8883702B883D
:1087E0001B0AC3702E8902250436F6B2F42E15D862
:1087F0001B4B9F4214D10C2002F0CAFF1135011E01
:108800000CD0902303708E3B0371043B4380154BC7
:108810008460C680187803F0D3F800252800FEBDD8
:108820005C237B43104AD3180093583301931B7881
:10883000002B0FD10300320038000099FFF742FFF0
:10884000019B05001B78002BE8D13800009903F04C
:1088500067F8E3E7054A0725536A01335362DDE70A
:10886000FEFF0000D865FF1F1466FF1FE065FF1FB5
:10887000F0B587B0009017200F0016000193FFF7A6
:10888000F2FD1325041E19D00C98031E02D0019985
:10889000201D9847030AE370052302AAA070043044
:1088A000908127700098667003A993800494FFF765
:1088B00087FF051E02D0200002F04AFF280007B003
:1088C000F0BD0000F0B587B01F000CAB1B78039122
:1088D000059301210DAB06001C78049200F0D6F838
:1088E0001425002821D02000FFF77EFD0135041E4D
:1088F0001BD01149059B0A7803700132D2B2131EB6
:10890000C68001D101231A000B7022713000049B34
:1089100003990097FFF7ACFF051E09D12300210042
:108920000648074A093303F08BF8280007B0F0BD6A
:10893000002363802370F8E7DC65FF1FBF8300110D
:1089400030750000F8B505000E00064C064F236890
:10895000002B02D03100280098470434BC42F6D1E5
:10896000F8BDC0468066FF1F9466FF1F0123064ABC
:108970005B425380002313715362044A13605360B7
:108980009360D360136170479466FF1F8066FF1F7A
:108990000200002310B506499C000859002801D1A7
:1089A000625010BD0133052BF6D11320F9E7C04604
:1089B0008066FF1F034A5388181A434258414042B9
:1089C000104070479466FF1FF0B585B002930AAB64
:1089D0001F780CAB1B88009008000E0001920393D7
:1089E000FFF7E8FF05001120002D1BD10E48FFF70F
:1089F000E1FF04001520002C14D006220B99A7716A
:108A0000E01D03F005F8019B30002371029B290053
:108A10006371009B66802370039B6562E381FFF7AF
:108A200091FF280005B0F0BDFFFF000010B5FFF773
:108A3000C1FF04000220002C12D060880121FFF742
:108A400081FF606A002801D002F042FE2822002146
:108A5000200002F0CDFF012300205B4263802071E3
:108A600010BD000030B5074A074C55880100137847
:108A70000020A54204D05B1A59424B415842104095
:108A800030BDC0469466FF1FFFFF0000084A10B5C6
:108A900001230C00904208D0FFF78CFF031E04D086
:108AA000037923405A1E9341DBB2180010BDC04623
:108AB000FEFF0000024B1879431E9841C0B2704778
:108AC0009466FF1F70B504000D001600FFF772FFDB
:108AD000002804D10D4B9C4200D0143070BD416A77
:108AE00003790520002907D012221A40102A02D14A
:108AF0000520002EF2D10F20DB06EFD5897E0C2059
:108B0000A9428941494249420840E7E7FEFF000087
:108B1000030010B5002800D110BD0348034A418866
:108B20009142F9D09847F7E79466FF1FFFFF0000D6
:108B3000002330B5C45CCD5C6C40D4540133102BA1
:108B4000F8D130BD0F23002210B5C45C640022436D
:108B5000CA54C25CD209013BF7D210BD0200010029
:108B600010B52032103102F0A3FD10BDF0B58BB06E
:108B70000390102005931700049102F0B1FD0090BE
:108B8000102002F0ADFD009B13240190002B05D0B6
:108B900000280CD11324009802F09AFD019B002BB1
:108BA00002D0180002F094FD20000BB0F0BD1020A0
:108BB00002F096FD0600102002F092FD132405003D
:108BC000002E00D1AEE0002819D01022002102F0C2
:108BD0000FFF32002900039802F06AFD041E0ED137
:108BE00033787F2B51D830000099FFF7ABFF009B03
:108BF0001B787F2B53D801990098FFF7A3FF300013
:108C000002F066FD002D02D0280002F061FD002C6C
:108C1000C1D1102002F064FD0600102002F060FDBA
:108C20000290002E7CD0002878D03A000F3223002A
:108C30000125121105D00F333B4015B25A42534162
:108C40001BB26A1E1201002B33D0049BD2B29818BB
:108C50000099029AFFF76CFF013D102200213000BD
:108C600002F0C6FEADB2049F2D017D19AF4242D085
:108C7000002C33D0300002F02BFD029B002B00D1E2
:108C800089E7180002F024FD85E729003000FFF78E
:108C900059FF28002549009AFFF74AFFA7E7290056
:108CA0000098FFF74FFF28002049019AFFF740FF87
:108CB000A5E70F210F4004998A18D9B28F4208D92D
:108CC000D15C06A819540133102BF6D1029A0199F0
:108CD000C0E7791A48424141C901F2E73900300042
:108CE00006AAFFF725FF3200039806A902F0E0FC70
:108CF00010370400BAE7002CBCD13000029906AA54
:108D0000FFF716FF320006A9039802F0D1FC0822F3
:108D100004003100059802F07BFEABE71324A9E7BD
:108D20001324AAE7002800D06EE733E7D0BE001175
:108D3000F0B58BB00F0016000225009000283FD040
:108D4000002A3DD00B1DDBB21800029302F0C8FCD4
:108D50001135041E34D0FDF747FD05003A00009997
:108D6000201D02F0ADFEEBB20393E3702B0CDBB2DF
:108D70002F0A00936370FFB22B0E2370A77001932C
:108D8000FDF72CFD1022010006A802F099FE21003B
:108D9000029A04AB06A8FFF7E9FE051E0DD1039B5E
:108DA00008223370009B04A9B370019B7770F370A5
:108DB000301D02F085FEFDF71DFD200002F088FC4D
:108DC00028000BB0F0BDF0B58FB00D00149E0390DD
:108DD00004920593002A03D1022420000FB0F0BDB5
:108DE000002EF9D00398FFF7E5FD1424071EF4D0F8
:108DF0007278337812021A43B3781B041343F27863
:108E000012061A43036A0192934201D30133E3D15C
:108E1000002D03D03B7901249B07DED508220021D9
:108E200006A802F0E5FD059B13240433DBB218000D
:108E3000029302F055FC051ECFD0059A0499043028
:108E400002F03EFE04223100280002F039FE390013
:108E5000102210310AA802F033FE2900029A06AB54
:108E60000AA8FFF783FE041E0FD1082206A908A84E
:108E700002F026FE0822311D08A802F061FE01283A
:108E800007D101990398FDF7C9FC280002F020FCE6
:108E9000A3E70124F9E7000070B51C4C0500236826
:108EA000181E10D0002D14D11A78002A0CD1981C4D
:108EB000083202F0ADFD02F05BFE0135002808D15A
:108EC00023681D70012070BD0A331800082202F0CB
:108ED0009FFD2368002BF5D0122002F059FC061EDE
:108EE0000DD0C12321680370457002311022023079
:108EF00002F08EFD23683100587802F061FD206891
:108F000002F0E6FB00232360DCE7C046BC66FF1FDF
:108F1000F8B504002020FDF755FB0D4EA700BB5906
:108F20000500002B0DD000280BD0D878FF2809D1E0
:108F300008492A000C55F35907480333611802F019
:108F40007FFDF8BD290002F09BFD0028F0D1F8E775
:108F5000D866FF1FC066FF1F69A1001170B5064DDE
:108F600084006359002B05D0D87802F099FCFF22C9
:108F70006359DA7070BDC046D866FF1F70B5060031
:108F80008CB00C00150000213022684602F030FD44
:108F900031001022684602F093FD1D2021000322BB
:108FA000684402F08DFD6846FFF7D8FD2D210400CE
:108FB00003222800694402F083FD20000CB070BD3C
:108FC000F0B50700160097B001931CAB1D78302256
:108FD0001EAB00910AA800211C7802F009FD1022A6
:108FE00039000AA802F06CFD1022002102A802F04C
:108FF000FFFC0722310002A802F062FD072202AB4B
:109000009818631E9C41019902F05AFD02AB9C73B3
:109010002B005A1E934102AAD3730021102206A8E6
:1090200002F0E6FC06221D9907A802F049FD1A206D
:1090300002ABC01806221F9902F042FD10220099CF
:109040000EA802F03DFD102202AB0EA908781C7894
:10905000013A6040D2B2087001330131002AF5D1E3
:109060000AA8FFF77BFD102212A904000EA802F047
:10907000CFFC102206AB0EA908781D78013A684093
:10908000D2B2087001330131002AF5D10AA8FFF7E6
:1090900065FD044310222098E4B212A902F010FDED
:1090A000200017B0F0BD70B50E0014008CB00100A8
:1090B000102268461D0002F003FD3100082204A8BA
:1090C00002F0FEFC2100082206A802F0F9FC684626
:1090D000FFF744FD04001022280008A902F0F0FC6C
:1090E00020000CB070BDF8B506000D000024371943
:1090F000AC4200D3F8BD02F053FB030A3B70631C83
:10910000DBB201379D4203D90234F054E4B2EEE7FA
:109110001C00EDE773B506000C000225002819D0ED
:10912000002917D0032101A8FFF7DDFF6B469A79CC
:109130003F231A40013313436A463000937101A95B
:109140002200FFF71BFF051E04D10322E01C01A92A
:1091500002F05EFC280076BD03785807DA08C00FDD
:10916000D20080009B0710439B0F1843C0B270478A
:1091700007230B40C908C9000B4303707047000068
:1091800070B50400FFF7EAFE134DA4006359002BED
:1091900021D0186A002801D002F09AFA2B59986E53
:1091A000002801D002F094FA2B59D86E002801D083
:1091B00002F08EFA2B59186F002801D002F088FABD
:1091C0002B59586F002801D002F082FA285902F07A
:1091D0007FFA00232B5170BDD866FF1F0E4B800015
:1091E000C35870B50C00002B0FD09D68002D0CD01B
:1091F0002B78201D0B706B784B70A97CFFF7B8FFA4
:109200002B7E23726B69E36070BD10220021200069
:1092100002F0EEFBF8E7C046D866FF1F014B18606E
:109220007047C046D466FF1F074A0300800082587B
:1092300010B5002A06D0D088984203D1012901D167
:10924000FFF79EFF10BDC046D866FF1FF0B5264E43
:1092500095B087000B93BB590500099112200A9223
:10926000002B31D0D888FFF7A5FB04001420002C78
:109270002AD0280010A9FFF7B1FFBB591E781D6A3C
:10928000002E23D00895FDF7EFFA07000020FDF728
:10929000F1FA0790A379E61D069310AD0CA9089882
:1092A00000F0E2FA0EA9280000F0D7FA0B9B0A9909
:1092B0000493069B09980293079B039601930097DA
:1092C0000EAB0CAAFFF77CFE15B0F0BDFDF7CCFA93
:1092D00006903000FDF7CEFAE31DA779079310AB97
:1092E00006000893DAE7C046D866FF1F30B50C4C7D
:1092F00085002A59030085B00120002A0ED01800ED
:109300006946FFF76BFF2B591A78D888054B002A5E
:1093100000D1054B6A46072100F0D9FB05B030BDEE
:10932000D866FF1F5B9800116998001130B5094C91
:109330008500295985B010226846253102F068FB66
:109340002A591121044BD0886A4600F0C0FB05B0B1
:1093500030BDC046D866FF1F0599001130B5094CD5
:109360008500295985B010226846353102F050FB3E
:109370002A591121044BD0886A4600F0A8FB05B099
:1093800030BDC046D866FF1F43990011F7B54D4F59
:1093900086001020F4590D0002F0A2F9F359206262
:1093A000186A132200286CD0033A29009C6802F046
:1093B0002FFBF3591A780192002A58D11E6A227D98
:1093C000317B944651400122019F114201D16746F1
:1093D0001740217D914339432175377B4F40BC466F
:1093E00060460027800701D44F0817400121022062
:1093F0008F40227D82433A432275377B5740BC46DB
:1094000060460027400701D497080F400420227DC2
:10941000BF0082433A432275627D0027944660462E
:10942000727B42400A4201D167460F400121627DB2
:109430008A433A436275777B5740BC4660460027B3
:10944000800701D457080F400220627D7F008243CD
:1094500017436775767B00227E40760701D4BA08F1
:109460000A400426617D9200B1430A4362756A781E
:10947000002A08D06278002A05D005220533DA7761
:1094800000221000FEBD04222979114205D1A17CE1
:10949000114202D10533033AF1E7019A21782C7881
:1094A000002A02D10A002100140018220429E8D859
:1094B000042CE6D805206043034A05331218525C99
:1094C000DDE7C046D866FF1FE0BE001110B50A00F8
:1094D0001121024B00F0FBFA10BDC0469F9900110C
:1094E0000B0030B587B001AD2B806B460400110036
:1094F000981D082202F08CFA2A000B212000024B52
:1095000000F0E5FA07B030BDC799001110B50A00A8
:109510001121024B00F0DBFA10BDC0461B9A00116E
:1095200013B50B0011006A4613706B460400062247
:10953000581C02F06DFA6A4608212000014B00F029
:10954000C6FA13BD3B9A001110B50A001121024B57
:1095500000F0BDFA10BDC0468B9A00117FB5050022
:109560000B4BAA00D4580800002C0FD0666F237F45
:10957000E28821780396266F0296E66E0196A46E25
:109580000094FDF709FC2800FFF7FAFD7FBDC046F7
:10959000D866FF1F10B51721FFF7E0FF10BD0000D0
:1095A00070B50A000D00064B0221040000F08FFA8E
:1095B000060029782000FFF7D1FF300070BDC046BB
:1095C0006B99001170B586B000236A4613708368EA
:1095D00004001D78681E0A2859D801A902F0E8FA8B
:1095E000060633373B3F43474B4F5300180000F00C
:1095F00042F9062312284BD000281BD16088FFF7C0
:10960000D9F90823002813D04279002A47D1264BE4
:109610001A78072312070BD5244B1A680723002A50
:1096200006D01668002E03D0290001AAB047030017
:109630006A4613706B461B786088002B2AD1FFF7AF
:1096400067FC06B070BD180000F06CF9D4E7180094
:1096500000F087F9D0E7180000F093F9CCE7180084
:1096600000F0ADF9C8E7180000F0C3F9C4E718002E
:1096700000F0F6F9C0E7180000F0F6F9BCE71800B2
:1096800000F013FAB8E7180000F013FAB4E7072364
:109690006A46137069466088FFF782FFD1E70523A9
:1096A000012AC5D1024BB8E76565FF1FD066FF1FD1
:1096B000D466FF1FF8B52C4F8600F35904000D0047
:1096C000002B40D0DA8882423DD15A78062A33D125
:1096D0001A78002A2ED0012099681A6A097D014261
:1096E00006D0157B054203D007225A700120F8BD31
:1096F0000220014204D0157B054201D00922F4E783
:109700000420014204D0127B024201D00B22ECE77C
:10971000164B1B68002BE9D05B68002BE6D02000BD
:109720009847BB5900215B78122BDFD12000FFF74F
:1097300015FFDBE70E4BECE7112A04D1002900D01E
:1097400032252900F2E7002D08D12000FFF732F979
:10975000002803D01023027913430371210028004D
:10976000FDF798FAC2E7C046D866FF1FD066FF1F14
:10977000D466FF1F70B50E4E8500AB590400002B58
:1097800013D01B78002B11D10A4B1B68002B04D07F
:109790005B68002B01D02000984773595B78122B2F
:1097A00003D100212000FFF7D9FE70BD024BECE78A
:1097B000D866FF1FD466FF1FD066FF1F094B8000CD
:1097C000C3581020002B0CD01A6A002A09D09B68BD
:1097D000002B06D0127A1B7E101C9A4200D9181C4E
:1097E000C0B27047D866FF1F70B503000D001400AB
:1097F0000220002A30D000292ED013700B78081DCB
:1098000053704B789370FFF7A7FCE07001200221A2
:109810002B7A23716B7B034063716A7B0A4013438D
:10982000042263716E7B1640334363716E7BF608CE
:10983000F600334363712B7B0340A371287B014007
:1098400000200B43A371297B0A401343A3712A7B99
:10985000D208D2001343A37170BD10B50A000100F5
:109860000120FFF7C1FF10BD10B50A000100022062
:10987000FFF7BAFF10BD70B506000C000220002EE5
:1098800030D000292ED07378201D0B70B3784B7028
:10989000F178FFF76DFC01223579257271794B1053
:1098A000080013409340104003438810104080008C
:1098B000C9080343C9000B436373B1794B10080017
:1098C0001340934010400343881002409200C9089F
:1098D0001343C9000B4321202373FCF773FE854219
:1098E00001D2122070BD2220257AFCF76BFE854242
:1098F000F7D823781820042BF4D86378012BF1D8FB
:109900000020EFE7030010B50220002909D0002B4A
:1099100007D00322481C0A7019000D3202F078F8B3
:10992000002010BD03000222080010B5002B06D055
:10993000002904D00E32591C02F06AF800221000EF
:1099400010BD030010B50220002909D0002B07D05C
:109950000422481C0A7019000C3202F059F8002049
:1099600010BD10B5FFF7DEFF10BD03000220002977
:1099700006D0002B04D0052200200A701B784B7003
:10998000704703000220002B08D0002906D05B7826
:1099900000200B70013B082B00D9183070470300E2
:1099A00010B50220002909D0002B07D00622481C40
:1099B0000A7019000A3202F02BF8002010BD10B511
:1099C000FFF7B0FF10BD02000B00022010B5002908
:1099D0000ED0002A0CD007211970118859701188F7
:1099E000090A997011180822D81C02F011F80020F9
:1099F00010BD03000A00022010B5002B0CD0002976
:109A00000AD099785878090201431180901CD91C1A
:109A1000082201F0FDFF002010BD030010B5022058
:109A2000002909D0002B07D00822481C0A70190011
:109A3000921801F0EDFF002010BD02000B00022083
:109A400010B500290BD0002A09D00921197011780E
:109A500018185970511C062201F0DAFF002010BDC1
:109A600010B5FFF75FFF10BD02000B00022010B51C
:109A7000002A09D0002907D0517819701118062240
:109A8000581C01F0C5FF002010BD030010B50220D6
:109A9000002909D0002B07D00A22481C0A7019009F
:109AA000063201F0B5FF002010BD10B5FFF73AFFF8
:109AB00010BD02000B00022010B5002A06D00029BC
:109AC00004D018005178FFF753FB002010BDF0B50B
:109AD00085B017001E006A46062305000800918124
:109AE0009380FEF7C0FC1324011E02900CD03800B6
:109AF000B047041E05D1280001A9FEF76FFA041E25
:109B000002D0029801F024FE2800FFF701FA20009D
:109B100005B0F0BDF0B504008BB001911500002137
:109B2000102202A801F064FF334EA700B8590028A4
:109B30003CD0C388A34239D10378002B36D1427878
:109B4000062A18D102000100553235310C3006AB1F
:109B5000FFF7A9FA002829D12000FFF72FFE020005
:109B600006A902A801F054FF200002A901F0E8FDB7
:109B700001200BB0F0BD816E002917D00B8A112A8D
:109B800028D19D420ED101981231093A01F0D8FF37
:109B9000012807D1BB5920009D6EFFF70FFE290059
:109BA0000200DEE732212000FFF7D8FC2000FEF79C
:109BB00001FF061E1BD0416A002918D00B8AAB4258
:109BC00015D108220198123101F0BAFF01280ED1F7
:109BD000716A0AE09D42E9D108220198123101F030
:109BE000AFFF0128E2D1BB59996E8A7EB9E7200008
:109BF00001F04EFDBCE7C046D866FF1FF0B56B4DC7
:109C000087007E5985B0337802900393002B00D0F3
:109C100087E0B368346A01937078062817D101226F
:109C20001B7D134202D0217B114218D10222134224
:109C300002D0217B114251D10422134203D0237B55
:109C4000134200D08BE0019B5A7DEB5991E007381D
:109C50000428F8D801F0ACFF032E42678300B36EEE
:109C6000002B03D11C2001F03BFDB066EB599C6E2C
:109C7000002C1CD010220021200001F0B9FE029817
:109C8000FFF79CFD01002000FFF72DFA01F088FD91
:109C90002082200008211230FFF725FA0298FFF7F2
:109CA0008DFDA076EB592100D888FFF70FFC082224
:109CB000EB591CE0B36E002B05D01A00198AF0880E
:109CC0001232FFF70DFC0222019B197DEB59114264
:109CD0003DD0207B10423AD0073208E0F488FCF7F0
:109CE000DBFD01002000FFF711FC0A22EB595A703E
:109CF000029B9C002A595378073B042B11D8D0882B
:109D0000FEF758FE00284ED0C3895A08D2182849B9
:109D1000029B0298CB542B5941180433254801F07B
:109D20008FFE05B0F0BDFCF79FFD030001208342CC
:109D300001D100200393EB59DE88FCF79BFD0399CA
:109D400002003000FFF7ECFB019AEB59117D042271
:109D500011420CD0217B114209D00B22C7E7F688B3
:109D6000FCF73CFD01003000FFF7EEFB6BE7019ACA
:109D7000527D01210A4204D0607B084201D00C22AE
:109D8000B5E702210A4204D0607B084201D00E22CE
:109D9000ADE704210A4204D0627B0A4201D01022BE
:109DA000A5E71222A3E7FA225200B0E7D866FF1F08
:109DB000DC66FF1F73A1001110B5064B1A7804234F
:109DC000100018401A4200D00348FFF727FA00207D
:109DD00010BDC0466565FF1FFC43FF1F70B5040042
:109DE000FFF7D4FA051E43D12000FFF77FFA234E78
:109DF000A400A0598268937CDB0708D50321036A7D
:109E00001B790B40012B02D1017F0B430377431DCC
:109E1000D97F8B1E022B0DD8022900D00121C088CA
:109E2000FCF790FF042133591A7F59700A431A77BF
:109E3000280070BD01290CD102231022437000219B
:109E40000C3001F0D5FD305910213530FFF74BF9BA
:109E5000EEE70529ECD10223D118437010220C3013
:109E600001F0D6FD04233259117F0B431377EAE743
:109E700008251828DCD1053DDAE7C046D866FF1F63
:109E8000F0B58BB0059143887E4F9E00F4591500C4
:109E90000493002C15D1012902D000200BB0F0BD95
:109EA000101D57781678FFF757F9EB6832000293C8
:109EB0002B7A0499019300903B002000FCF70CFFE3
:109EC000EBE7E388049A934201D00820E6E7237881
:109ED000012B00D1D4E0059B581E092800D9CFE002
:109EE00001F066FE05CE0A29CC506C859AB2290095
:109EF0000498FFF773FFD1E72000290010224530B6
:109F000001F086FDB9594B78042B02D1013B4B700F
:109F1000C3E70B000A00253335320C310498FFF7F4
:109F200095F90498FFF702FA0522431E9841BB59A0
:109F3000C0005A70B2E7200029001022553001F00D
:109F400067FD049B4F4C9D00295904980A0006ABFD
:109F500055320C31FFF77AF929591022453106A8FC
:109F600001F0EEFD012808D10498FFF7F7F90590FC
:109F7000002804D106222B595A7005988EE7082331
:109F80000593FAE763780C2B7AD1E36E002B03D1AB
:109F90001C2001F0A5FBE066BB59D86E00286FD0ED
:109FA0001022290001F034FDBB590498DC6EFFF744
:109FB00005FC0D22A076BB595A706EE7E06E0028B2
:109FC0005ED063780D2B5BD12B8808220382A91CFD
:109FD000123001F01DFDBB599A68517D02221142D9
:109FE00026D0186A407B104222D00C32E4E7637816
:109FF0000E2B45D1236F002B03D1162001F070FBEF
:10A000002067BB59186F002803D01022290001F0E7
:10A01000FFFC0F22BB59CFE763780F2B30D1206FA5
:10A020000622691C103001F0F3FCBB599A68517D7F
:10A030000422114203D0196A497B1142D5D1002173
:10A040000498FFF78BFA28E7636F002B0DD0BB59FC
:10A05000586F0028F3D01022290001F0D9FC01220A
:10A06000BB5952425B6F1A61E9E7142001F038FBDB
:10A07000BB5960675B6F002BE9D126E72978DFE7E2
:10A0800007200BE7D866FF1F10B5064C207001F0C3
:10A0900077FD06212078FDF791FF0348FEF778FC55
:10A0A00010BDC046EB66FF1F2992001100200BB2C5
:10A0B00070B50D00834216DA264B187801F0B0FB1C
:10A0C000041E0DD00378922B0ED0A02B37D0224B3C
:10A0D0001878FF283AD0210001F072FC002835D111
:10A0E00080200002684070BD43780E2B0BD03E2BC1
:10A0F000EDD18378052B12D0082BE8D181798088A7
:10A10000FFF7D8FA08E0154B82889A42DFD18368BE
:10A110001878591CFEF7C0FE002817D1D7E7104B5E
:10A120001B785B0712D50F4B1B68002B0ED09B686A
:10A13000002B0BD0C289811D80889847ECE7FFF780
:10A1400041FAA068002801D001F002FB200001F0D4
:10A15000A7FAC5E7EB66FF1FF543FF1F18200000B5
:10A160006565FF1FD466FF1F10B50078FFF712FA70
:10A1700010BD10B50078FFF7FDFA10BD0C23434366
:10A18000084A10B59B185A68002A03D0012901D14A
:10A19000904710BD9B68002BFBD00029F9D1984750
:10A1A000F7E7C0460867FF1F01238340094A10B53F
:10A1B000946B1C439463506B98435063D46B2000A2
:10A1C0009843012901D120001843D063116B0B4340
:10A1D000136310BD00800040F0B500240127154B2B
:10A1E00085B0DA6B144E03921A6C0192DA64019B0B
:10A1F000E3403B4217D0039DE5403D400295E5B268
:10A2000002992800FFF7BAFF316A736A002908D063
:10A210003900002B01D0029979402800FFF7C4FFD4
:10A2200001E0002BF9D101340C36172CDFD105B039
:10A23000F0BDC04600800040EC66FF1F064B0121C8
:10A240005A68C2400A4204D01B68C3401800084044
:10A2500070471B6DF9E7C046008000400122064BA5
:10A260008240002903D0D9680A43DA607047D96870
:10A270009143D960FAE7C0460038004030B5032466
:10A2800044430F4BE25C1B199C785D7801232D1B26
:10A290000135AB40013BA340A140DB430C00122839
:10A2A00007D80849920052181168194021431160DB
:10A2B00030BD054A11680B4023431360F8E7C046E0
:10A2C00027BF001108F0004014F00040C21F70B515
:10A2D000D4B20623092C0BD80125084C954000293F
:10A2E00008D00021FFF7CAFF23682B432360002317
:10A2F000180070BD2368AB43F8E7C0460038004043
:10A30000214BF0B51B185B78022B21D10324444369
:10A310001E4A1F4EA35C1219947801221500854035
:10A32000B76B013CE4B23D43A240B563194C12281F
:10A3300015D89B0000290CD117495B1899680A436E
:10A340009A600123205C154A834011680B43136017
:10A35000F0BD11495B18996891439960F1E70E4B84
:10A3600000290DD159690A435A61225C1328E8D0AB
:10A370000123203A93400A49086803430B60E7E74A
:10A38000596991435961F0E7EC66FF1F27BF00113F
:10A39000008000406CBF001100F00040A0F00040C1
:10A3A000A4F00040F8B500241B4E1C4D1C4B1B5D57
:10A3B000012B1FD1194A9269E2401A420BD00122A7
:10A3C000B25693402200143AD2B2022A09D8154953
:10A3D0004A6913434B61013402360C35172CE5D121
:10A3E000F8BD0022B2560F499200521891680B43F3
:10A3F0009360F0E7022BEED1E7B23800FFF71EFFC3
:10A4000001235840C1B23800FFF77AFF3800FFF748
:10A4100015FF6877DFE7C046F9BE0011EC66FF1F45
:10A42000ED66FF1F00F00040012202388240054B1C
:10A43000002903D059690A435A6170475969914309
:10A440005961FAE700380040F8B50E0001210F000D
:10A450008740114A0400D368FD43BB43D360831E89
:10A460008B4201D8FFF7E0FF00212000FFF72EFF0D
:10A470000A4A0B4B5168012E05D139431B19516013
:10A480005E700020F8BD2940516002221C196270E4
:10A490009A6915409D61F4E7003800400080004053
:10A4A000EC66FF1F012210B58240074B002906D041
:10A4B00019680A431A600121FFF7C6FF10BD196829
:10A4C00091431960F7E7C046008000400C2370B547
:10A4D000002543430A4A29009B181D70094B0400BC
:10A4E0001B185D70FFF7B0FF0123A3400649280049
:10A4F0000A681A430A6005490A689A430A6070BDEF
:10A500000867FF1FEC66FF1F34800040308000406A
:10A5100070B504000E00FF2813D003250540FFF797
:10A52000D5FF084AA3089B009B183F22ED00AA40D4
:10A53000AE40196820009143314319600121FFF7B3
:10A540008DFE70BD18380040F8B50C244443134B01
:10A550000500E4186368002B03D1A3681220002BC8
:10A560001AD0022201270E4B00215B195A702800D5
:10A570002770FFF769FF63681E1E08D0A3683E00BE
:10A58000002B04D02800FFF759FE4640F6B2280001
:10A590003100FFF709FE0020F8BDC0460867FF1F25
:10A5A000EC66FF1FF7B5C420FF222B4B8000195823
:10A5B000002491433F3A0A431A508022274F520207
:10A5C000274E1A60274B1D5D002D21D0A31E012BA5
:10A5D00003D80121E0B2FFF727FF012D18D11F4B4F
:10A5E0009B69E3402B4213D0E3B218000193FFF7BD
:10A5F00025FE01000198FFF755FFE3B2143B022B43
:10A600001DD801217156184A8D405369AB435361DF
:10A610003B7F002B0DD0E5B22800FFF795FF280007
:10A62000FFF70CFE7B7F0100834202D02800FFF77A
:10A63000A5FD01340C370236172CC3D1F7BD01211B
:10A6400000237156F3568D40074A9B009B189A6869
:10A65000AA439A60DCE7C04600E100E0EC66FF1F19
:10A66000F9BE0011ED66FF1F00F0004070B50E004E
:10A6700015000400FFF72AFF0C236343094A20005A
:10A680009B189D605E60FFF75FFFF021064B074A55
:10A690008900051E5A5002D02000FFF717FF28003E
:10A6A00070BDC0460867FF1F0000FF1FD9A1001141
:10A6B00070B5134D07202C78002C1FD19822210053
:10A6C0005200280001F09CFA0123C420FF222B70C5
:10A6D0000C4B80001C635C630B4B1C605C600B4B81
:10A6E000195891433F3A0A431A50802252021A6085
:10A6F0000D20074A074900F0A3FF200070BDC046A7
:10A70000EC66FF1F00800040A0F0004000E100E088
:10A71000A5A50011A5A30011030010B50620072B65
:10A7200009D8054A137001F07BFAD7210020034BAA
:10A73000034A89005A5010BD2444FF1F0000FF1F28
:10A74000951BFF1F70B51D0002240C2910D8094A63
:10A75000CA40D2070CD5FBF741FF041E08D1059A69
:10A7600004992800FBF756FFFCF7C4FDFFF724FB14
:10A77000200070BD1210000030B50D7802232C00AF
:10A780009C43184201D02B431C0008252300AB43F7
:10A79000284201D02B00234320241D00A543204242
:10A7A00001D01C4325002A230D70184204D01178D3
:10A7B0001E3B0B43137030BD0028FCD10C211378D5
:10A7C0008B43F7E7F8B51D0006AB1B88140007AAFA
:10A7D0000E000B201778002B27D10A78022A49D1C6
:10A7E0004A68507811780002244A084380180428E7
:10A7F00040D801F0DDF903121D1B2300F06800F0C2
:10A800005FFF021CC0B2B84200D93A1CD2B220008D
:10A81000F1682A8001F0FCF806E00222F3681B8848
:10A820002A8023701B0A63700020F8BD0622EEE721
:10A8300001232B80F3681B782370F5E7F368002B66
:10A8400016D008222A801A8822701A88120A62708A
:10A850005A88A2705A88120AE2709A8822719A88DD
:10A86000120A6271DA88A271DB881B0AE371DBE7E6
:10A870002B80D9E701202B80D7E7C04600D6FFFF09
:10A88000F7B516000A781D0008AB1F880C000123DD
:10A89000022A18D14A685078117800022B4A0843DE
:10A8A000801803280FD801F083F902254439E068A5
:10A8B00000F006FFC0B20723B84204D37B1901930E
:10A8C000152B02DD0D231800FEBDE0682A003100C3
:10A8D000C01901F09DF86B4600209B88E268D054B7
:10A8E0001B4B1B68834203D01B68834200D09847F0
:10A8F0000023E8E70B23002FE5D1022DE2D1737886
:10A9000032781B021343E2681380114B1B68002B43
:10A91000EED01B68002BEBD00120E8E70B23002FC3
:10A92000D1D1062DCED12A003100E06801F070F8B7
:10A93000DEE70B23002FC6D1012DC3D1327875334A
:10A94000012AC0D8E3681A70D2E7C04600D6FFFFDC
:10A95000F868FF1F70B50C001500072837D801F004
:10A9600027F9041436361B36242E182015290BD847
:10A97000184E16220021300001F03AF8220029007A
:10A98000300001F045F8002070BD18200229FBD1ED
:10A990001288114B1A80F6E718200829F4D10A0012
:10A9A0000E48290000F01CFFEDE718200129EBD12B
:10A9B0000B4B10780B49DA69FFF7DEFEE3E718204E
:10A9C0000129E1D1064B10780749DA6BF4E7022040
:10A9D000DAE7C046E068FF1FA244FF1F9844FF1F4C
:10A9E0002844FF1F5044FF1F7044FF1F030010B591
:10A9F0000020DB0704D50721024A034800F08CF849
:10AA000010BDC04684BF00112844FF1F054A030043
:10AA10001068002803D082889A4201D1806870476C
:10AA20000068F6E7F06AFF1F0A88030008009A42F0
:10AA300004D08A8804309A4200D000207047000079
:10AA4000F8B5F22200230D4F0D4E79680500424300
:10AA50003370994200D07B600A4C0021200000F046
:10AA6000C7FF00231A007C60AB4202D10020337084
:10AA7000F8BD01332280DBB2F234F5E7E86BFF1F4B
:10AA8000E66BFF1FF46AFF1F73B56B46019006006B
:10AA9000684615001980FCF75FFF041E11D1002DD8
:10AAA0000FD07689002E11D00C2000F019FE00285E
:10AAB0000ED0084A0460136886808560002B02D19E
:10AAC0001060200076BD1A001B68F7E70224F8E743
:10AAD0001324F6E7F06AFF1F012100220A4B10B58C
:10AAE00049420A4C198099809A719A70084B2070DB
:10AAF000012019805A60FFF7A3FF2078FCF78AFF36
:10AB00000448FDF745FF10BD0069FF1FF06BFF1FF4
:10AB1000E86BFF1FC5AB0011022310B5002802D05F
:10AB2000FFF7B2FF0300180010BD0000030010B5CE
:10AB30000020DB0704D50421024A0348FFF7A4FFE5
:10AB400010BDC04698BF0011A844FF1FF0B50E26E7
:10AB500087B003930CAB1F8802ABF6180500080002
:10AB600031000292FDF77AF804000120002C0FD08A
:10AB70003088FFF74BFF03000E20002B08D05E68E3
:10AB8000002E05D021002800039B029A0097B047B1
:10AB900007B0F0BD0A4B10B5984207D1012200233F
:10ABA00052420A808B708A808B7110BDFFF73CFF88
:10ABB0000028FAD001235B42038000238370F4E76E
:10ABC000FFFF0000F8B5050001290AD1134E00244B
:10ABD0003388F227AB4219D028001149FFF7DAFF7A
:10ABE00006E0022904D10139FDF750FF0028EDD01D
:10ABF000F8BD3B0063437268D018D35A002B09D0CC
:10AC00003A00002100F0F4FE0134E4B2054B1B7859
:10AC1000A342EED801235B423380DDE7E86BFF1FE0
:10AC20000069FF1FE66BFF1F10B5FFF7FDFE030075
:10AC30000020834200D0987810BD0000F0B589B0A4
:10AC40001C000EAB80CB03901E8810AB1B780492C7
:10AC500002930B7A0D00DB0616D42B780593022B9A
:10AC600024D00498FFF7D2FE002812D003689C4637
:10AC7000002B0ED0029B2200019329003B0064466A
:10AC800003980096A04705E00498FFF7BFFE002850
:10AC900002D10E2009B0F0BD8368002BF9D00A2242
:10ACA0002900039898470028D7D0F3E76B685878B5
:10ACB0001A786B4B000210439842D2D8043B98425A
:10ACC00010D2684B984242D015D8674BC018012863
:10ACD000C7D80B20002EDDD1EB681A7859683A806E
:10ACE000200028E0614BC018032800D979E000F06B
:10ACF0005FFF846A789E5E4B9842B2D10B20002E93
:10AD0000C8D101233B80EB6831001B782370688930
:10AD1000013080B2FCF7A2FF3A88031E0ED0017802
:10AD200002328A183A80428962704289120AA270FD
:10AD300059680278E01C00F06BFE06E004323A80AD
:10AD400031000422601C00F053FE0020A2E70B201B
:10AD5000002E9FD1EB6807A91E8804233B80330A8D
:10AD6000300026706370FCF779FF051E28D004AB15
:10AD70009A890E2304A95B183E49C668FCF7E2FFD6
:10AD800000280BD12B783C486A680599FBF798FBA3
:10AD9000002803D1012304AA5B42D3813278022A1E
:10ADA00006D17168201D00F033FE3B8802333B80E2
:10ADB0000E2304AA9B181B88A3701B0AE370C4E728
:10ADC00004ABDE81F4E70B20002E00D062E7E968D7
:10ADD0000398FFF729FF02233B802070000A607070
:10ADE000B3E70B20002E00D054E70222EB681B884B
:10ADF0003A8023701B0A6370A7E7E86800F060FCE4
:10AE0000C2B203000720B24200D243E70DD002993C
:10AE1000DBB27118994202DB921BD3B20293029B00
:10AE2000E9681A003B8089195AE70023F6E70B20EE
:10AE3000002E00D02EE70722EB683A801A782270A5
:10AE40005A7862705A88A2705A88120AE2701A7987
:10AE50002271DA886271DB881B0AA37175E7C0462C
:10AE6000042900000228000000D8FFFFFFD6FFFFE2
:10AE700003280000FFFF0000C8BE0011F0B58DB030
:10AE80006B460020089120229B5E83423DDAA64B50
:10AE9000187800F0C5FC071E32D00378B02B2CD1F7
:10AEA0000079023816281FD800F0E2FD17001E00B6
:10AEB0001E001E0031001E0096001E001D011E0017
:10AEC00052011E0073011E00CD011E0050021E0023
:10AED0001E001E008E021E00E302944B94491B8844
:10AEE00078880B80FBF72CF83800FCF7ADFF914B0E
:10AEF0001B68002B01D038009847380000F0D0FBC9
:10AF00008020089B0002434018000DB0F0BDEE22E7
:10AF10000021874800F06CFD0BAA3B7B79893889BA
:10AF200000923A000D32FCF7B1FD0400804B1B7813
:10AF3000002C3FD146E0804B788805937F4B410041
:10AF4000CB5A0BAE073BDBB232880293002301934E
:10AF50007B4B210006930093059BFFF76FFE744D1A
:10AF6000002810D1069B3A8A1B889A420BD13800E0
:10AF70000599123000F0E4FD002804D02B78628996
:10AF80009B00EB185A80162306A81B183288200055
:10AF90007989FCF7D7FE2B7804009A00AA1851880B
:10AFA0000029C3D00133DBB22B70002807D006A9DB
:10AFB000C98A9180634A12889A42BCD802E0012172
:10AFC00049429180002B04D059497888FAF7ECFF68
:10AFD0008AE73E890A2479E000253E89574B06938B
:10AFE0007B88069A5B009B5A033B9D4202DB002D47
:10AFF000F0D05BE0162206A812183B7B79890092FC
:10B000003A0030000D32FCF741FD0590002858D081
:10B010004689017A7888FCF703FD041E44D1464B2B
:10B0200078880793069B4100C95A454B0439C9B239
:10B0300006AAD28A06930291019400930599079B70
:10B04000FFF7FCFD041E2FD1069B39491A88931C7B
:10B05000002D26D14B807988384B4900CB5A5119A5
:10B06000033B8B4220DD059B31485B8941190B7105
:10B07000A91C0135C9B2EDB2059145191B0A2B7106
:10B08000059B2D490433181800F0C2FC2C4B059A7F
:10B090001B88D318DDB22C4B9E4205D00136B6B2C8
:10B0A0009CE749889942D6D0002D0CD0204C28002E
:10B0B000618800F06DFC207021007888FAF784FF29
:10B0C00012E7059CF0E7002C00D183E77B78142B76
:10B0D00000D109E716493B794E800B700C717888D6
:10B0E000FAF724FF00E7162406ABE418210038899C
:10B0F000FCF7B4FD011E00D1B7E1788822880F4C1F
:10B1000045002C5B0A4D013CE4B2029400240F4B35
:10B1100001940095FFF792FD041E00D014E1290070
:10B120007888FAF761FFDFE6F06BFF1F9443FF1F9B
:10B130000869FF1FFC68FF1FFC69FF1F3865FF1FC0
:10B14000EC6AFF1F9243FF1FFFFF00000A69FF1F09
:10B15000162406ABE41821003889FCF77FFD011E98
:10B1600000D182E178882288AE4C45002C5BAE4D40
:10B17000013CE4B202947C89AC4B01940095FFF74A
:10B180005DFD041E00D0DFE029007888FAF736FF65
:10B19000AAE60025A44B1D803B00F6331B78A24A8B
:10B1A00078880792AB4208D99E4B1288069306997D
:10B1B00043005B5A013B9A4203DB0799FAF728FFE9
:10B1C00092E616246B00FB18059306ABE418059B6A
:10B1D00021001889FCF742FD011E03D1059B0124C3
:10B1E0001E8973E77888924B2288069C0993430056
:10B1F0001B5B904E013BDBB2029300230096019350
:10B20000099BFFF71BFD041E02D0059B1E895DE70D
:10B210007B88069A5B009B5A079A1088328812181E
:10B22000934202DC1B1A013B33807F4C0230328890
:10B230000999001900F0ECFB2388328801359B182E
:10B240002380EDB2A8E70BAA3B7B7989388900926D
:10B250003A000D32FCF71AFC00250590059B002BE7
:10B2600004D10A24002D00D16EE060E0059B7888AF
:10B27000197AFCF7D5FB0100041E63D1694C6C4BB5
:10B28000788806940993069B4400E45A694B063C6F
:10B29000E4B20BAE328807930294019100930599B2
:10B2A000099BFFF7CBFC041E4CD1079B5E491B8812
:10B2B0001A1D002D30D14A80059B5B4C5A896319B9
:10B2C0001A716B1C9BB2E318120A1A71162306A896
:10B2D00032881B1879890598FCF734FDFF21AA1CD8
:10B2E0002E1D03350B00059092B2B6B2ADB2002808
:10B2F00003D006ABDB8AD9B21B0AA21865191171FB
:10B300002B714C4D301D2A884949201800F080FBD4
:10B310002B88F618B5B2A1E74988914207D17A88FF
:10B3200006995200525AEB18053A9A42C4DC3E4C38
:10B330002800618800F03CFA207021007888FAF734
:10B3400071FED1E5002DF2D13E89BFE6162606AB8F
:10B35000F61831003889FCF781FC3D000400FA350D
:10B3600000282DD0037A9B060CD400227B893989D2
:10B37000788800923A000C32FFF7E8FB041E10D0E8
:10B380003E8915E03088FFF741FB00281AD083681A
:10B39000002B17D02100122278889847041EE4D091
:10B3A000EEE72B78002B02D17888FAF74BFE0026C7
:10B3B0002B78002B00D097E5002C00D194E585E692
:10B3C0000124DDE70E24DBE7162506ABED18290086
:10B3D0003889FCF743FC041E47D0037A9B0611D43E
:10B3E000154A7B881188994203D01448814207D1BD
:10B3F0001380134BF2261D780023D9B2A94221D322
:10B400000924A1E72888FFF701FB00282FD08368D3
:10B41000002B2CD02100122278889847041EDFD000
:10B4200092E7C0463865FF1F0869FF1F0A69FF1FC2
:10B43000FC69FF1FEC6AFF1FE86BFF1FFFFF0000A6
:10B44000E66BFF1F31005943546801336018615A9D
:10B450000029D2D13C0008342100F22200F0D8FAB1
:10B4600021007888FAF7F6FD3EE501246CE70E240A
:10B470006AE71D4B1A887B889A4231D07888FAF7A0
:10B48000F3FD31E5F223059851684343CD18C95ABD
:10B4900000291FD03B7A012B0BD16C88AB887888B0
:10B4A000AA1D0094FFF752FB041E02D000233B723A
:10B4B0002E88F2220021280000F09AFA00232B8027
:10B4C000059B0133DBB20593084B05991B78064AAF
:10B4D0008B42D7D801235B421380002CCED0F5E5F8
:10B4E000002634000596EFE7E86BFF1FE66BFF1FB1
:10B4F00070B504000E001500FFF796FA031E08D180
:10B5000031000548FFF790FA03001120002B02D00C
:10B510001C8000209D7070BDFFFF0000F8B50B4F30
:10B5200006003B780D001400FF2B0ED00A2000F01F
:10B530002FF9011E09D0B123038000234680037137
:10B54000C5800481387800F03BFAF8BDE944FF1F5C
:10B55000F7B50F0008A90600088809A90B24098877
:10B56000002821D10234022B1ED1557813782D02E8
:10B570001D432B008B4301937334002B14D1FB68C4
:10B58000300019000093FFF74FFB019C85420BD060
:10B590002A0030000099FFF7ABFF041E04D12A00F7
:10B5A00030007989FFF7BAFF2000FEBDF0B50E78B4
:10B5B00085B003900AA805880120022E0DD14C68A1
:10B5C0002778647824023C43054FBC4205D1039898
:10B5D000DBB201960095FFF7BBFF05B0F0BDC0469A
:10B5E00002290000034B10B51B68002B00D09847C0
:10B5F000FEE7C046F46BFF1F07B501A8FFF7F2FF97
:10B60000044A05480021121A00F0FAFAF8F7F2F895
:10B61000FEE7C046F86BFF1FEC44FF1F0000000070
:10B6200001B40248844601BC604700BFC9A90000BC
:10B6300001B40248844601BC604700BF55220000A7
:10B6400001B40248844601BC604700BF1D31FF1FA2
:10B6500001B40248844601BC604700BF156B01007D
:10B6600001B40248844601BC604700BF0939FF1F8E
:10B6700001B40248844601BC604700BFA54F0100E9
:10B6800001B40248844601BC604700BF8D1200002F
:10B6900001B40248844601BC604700BF091B00009A
:10B6A00001B40248844601BC604700BF434D01001D
:10B6B00001B40248844601BC604700BFE548000071
:10B6C00001B40248844601BC604700BFDD5201005E
:10B6D00001B40248844601BC604700BF014C010030
:10B6E00001B40248844601BC604700BF3D4B0100E5
:10B6F00001B40248844601BC604700BF2124000019
:10B7000001B40248844601BC604700BFED4A010015
:10B7100001B40248844601BC604700BF8552010065
:10B7200001B40248844601BC604700BFA93AFF1F2C
:10B7300001B40248844601BC604700BF8B5201003F
:10B7400001B40248844601BC604700BF311B0000C1
:10B7500001B40248844601BC604700BFD9490100DA
:10B7600001B40248844601BC604700BF456B01003C
:10B7700001B40248844601BC604700BF056A00006E
:10B7800001B40248844601BC604700BF4139FF1F35
:10B7900001B40248844601BC604700BF1D4D010052
:10B7A00001B40248844601BC604700BF2951010032
:10B7B00001B40248844601BC604700BF090E000086
:10B7C00001B40248844601BC604700BFC94A010079
:10B7D00001B40248844601BC604700BF055E00001A
:10B7E00001B40248844601BC604700BF810E0000DE
:10B7F00001B40248844601BC604700BF55490100BE
:10B8000001B40248844601BC604700BF8139FF1F74
:10B8100001B40248844601BC604700BF51250000C6
:10B8200001B40248844601BC604700BFF54E0100E8
:10B8300001B40248844601BC604700BFF30E00001B
:10B8400001B40248844601BC604700BF1534FF1FA5
:10B8500001B40248844601BC604700BF291C0000B7
:10B8600001B40248844601BC604700BF090E0000D5
:10B8700001B40248844601BC604700BF75A90000BE
:10B8800001B40248844601BC604700BFB3520100C6
:10B8900001B40248844601BC604700BFF538FF1F71
:10B8A00001B40248844601BC604700BF1147010053
:10B8B00001B40248844601BC604700BFF94C010056
:10B8C00001B40248844601BC604700BF6DBC000063
:10B8D00001B40248844601BC604700BF45500000E7
:10B8E00001B40248844601BC604700BF3D18000017
:10B8F00001B40248844601BC604700BF4D37FF1FBA
:10B9000001B40248844601BC604700BFADAE0000F0
:10B9100001B40248844601BC604700BF0138FF1FE4
:10B9200001B40248844601BC604700BF3919FF1FBB
:10B9300001B40248844601BC604700BF4D1F0000AF
:10B9400001B40248844601BC604700BFE117000013
:10B9500001B40248844601BC604700BF9530FF1F18
:10B9600001B40248844601BC604700BF7D36FF1F1A
:10B9700001B40248844601BC604700BF9DA9000095
:10B9800001B40248844601BC604700BF0D19FF1F87
:10B9900001B40248844601BC604700BF350E000078
:10B9A00001B40248844601BC604700BF350E000068
:10B9B00001B40248844601BC604700BFB54C010099
:10B9C00001B40248844601BC604700BF594F0100E2
:10B9D00001B40248844601BC604700BF5D17000007
:10B9E00001B40248844601BC604700BF2146010003
:10B9F00001B40248844601BC604700BF154D0100F8
:10BA000001B40248844601BC604700BF2D3AFF1FC5
:10BA100001B40248844601BC604700BFE94C010004
:10BA200001B40248844601BC604700BF7D30FF1F5F
:10BA300001B40248844601BC604700BF691F000092
:10BA400001B40248844601BC604700BFA94601001A
:10BA500001B40248844601BC604700BF352EFF1F79
:10BA600001B40248844601BC604700BFC51D000008
:10BA700001B40248844601BC604700BFFD3BFF1F84
:10BA800001B40248844601BC604700BF5147010031
:10BA900001B40248844601BC604700BF0D5201005A
:10BAA00001B40248844601BC604700BF4D36FF1F09
:10BAB00001B40248844601BC604700BF65710100C3
:10BAC00001B40248844601BC604700BF45510100F3
:10BAD00001B40248844601BC604700BFBD32FF1F6D
:10BAE00001B40248844601BC604700BFD53BFF1F3C
:10BAF00001B40248844601BC604700BFE928000049
:10BB000001B40248844601BC604700BF25260000FE
:10BB100001B40248844601BC604700BF5936FF1F8C
:10BB200001B40248844601BC604700BF595201007D
:10BB300001B40248844601BC604700BFC56D0100E6
:10BB400001B40248844601BC604700BFCD4C0100EF
:10BB500001B40248844601BC604700BFEDA5000067
:10BB600001B40248844601BC604700BFC139FF1FD1
:10BB700001B40248844601BC604700BFD91B0000E5
:10BB800001B40248844601BC604700BFC9260000DA
:10BB900001B40248844601BC604700BF7918000028
:10BBA00001B40248844601BC604700BFB14E0000AA
:10BBB00001B40248844601BC604700BFE93BFF1F57
:10BBC00001B40248844601BC604700BF851F0000E5
:10BBD00001B40248844601BC604700BFC521000093
:10BBE00001B40248844601BC604700BF812EFF1F9C
:10BBF00001B40248844601BC604700BF0124000034
:10BC000001B40248844601BC604700BFB70E000083
:10BC100001B40248844601BC604700BFE532FF1F03
:10BC200001B40248844601BC604700BF951BFF1F5A
:10BC300001B40248844601BC604700BF017F000098
:10BC400001B40248844601BC604700BFD53AFF1FDB
:10BC500001B40248844601BC604700BFDD660100B4
:10BC600001B40248844601BC604700BF355500005E
:10BC700001B40248844601BC604700BF1D4B01006F
:10BC80000003010302020303040205000602070089
:10BC9000080009020A030B030C000D000E030F033A
:10BCA000100311031300140015031603A13B001128
:10BCB000D53B00110000000002000000C2BC0011D2
:10BCC000192A0F180A000000F1590000FD24000095
:10BCD0004146010099800011ADA0001101750011CD
:10BCE0009D7E0011115300117DAE00115D4F0011BA
:10BCF000B13D0011E13E00110000000016160000E9
:10BD0000020000000CBD0011F4FFF3FFD2FC0000A4
:10BD1000214000110000000000000000547579610E
:10BD20000042312E34003030313800676974687554
:10BD3000622E636F6D2F70767678005448303544EC
:10BD4000000000000200000058BD0011292A282A26
:10BD5000272A262A252A242A0A180000E20400009D
:10BD60007102000078EC0000744000001027000011
:10BD700060F0000006640000204E0000000000009B
:10BD8000050000001F501D00023CB4000001180017
:10BD900014000000A1020000303132333435363750
:10BDA0003839414243444546000000001557001110
:10BDB000695700110000000002000000C4BD00111E
:10BDC0006F2A6E2A1A18EAD8BC80F0FC60000000C6
:10BDD0000000000000005F066B2F363D7D077F3FAF
:10BDE000777C596E7971AF066D4FC6CBEB0EEFCFF6
:10BDF000EEC3A966E9E8FA60D6F46CBCBEE0FEFCCE
:10BE0000EE3E9A769E8E000001A000000000000029
:10BE10006410B71DC8206E3BAC30D9269041DC764B
:10BE2000F4516B6B5861B24D3C7105502083B8EDF5
:10BE300044930FF0E8A3D6D68CB361CBB0C2649B19
:10BE4000D4D2D38678E20AA01CF2BDBDFB349B5F3E
:10BE5000800000800010000000000000036100115D
:10BE60008D77001127610011957B0011AB610011E6
:10BE70006B7B001121620011417B00117362001184
:10BE8000097D0011DB620011097D00110D630011B5
:10BE9000C37C001121620011F97A0011996200112E
:10BEA000A17C001100000000000000007F63001171
:10BEB000A17C0011E1630011A5770011052A042A75
:10BEC000012A002A02290328012800280118001845
:10BED00000000000000000000000000000000087DB
:10BEE0000101020102010102010203030401030135
:10BEF000010101010303020103000D000E00100007
:10BF0000110013001401070108010A010B011C01B3
:10BF10001D02040205020702080219021A021C028D
:10BF20001D030103020317000201000504000807B6
:10BF3000000B0A001716001D1C0102010105040177
:10BF40000E0D011110011413011716011A19020226
:10BF500001020B0A020E0D02111002141302171631
:10BF6000030504030807030B0A030E0D0001020377
:10BF700007090A0B0E0F101112141718191A1B1F9C
:10BF800020212200C5A7001181A800110000000097
:10BF900002000000CEBE001100000000ADB500118F
:0CBFA0000000000002000000CCBE0011F8
:020000041FFFDC
:1000000000000000193D0011C8BC0011C4BC001163
:100010001C62FF1F00000000000000000000000044
:1000200000000000000000000000000000000000D0
:1000300000000000000000000000000000000000C0
:1000400000000000000000000000000000000000B0
:1000500000000000000000000000000000000000A0
:100060000000000000000000000000000000000090
:100070000000000000000000000000000000000080
:100080000000000000000000000000000000000070
:100090000000000000000000000000000000000060
:1000A0000000000000000000000000000000000050
:1000B0000000000000000000000000000000000040
:1000C0000000000000000000000000000000000030
:1000D0000000000000000000000000000000000020
:1000E0000000000000000000000000000000000010
:1000F0000000000000000000000000000000000000
:1001000000000000000000000000000000000000EF
:1001100000000000000000000000000000000000DF
:1001200000000000000000000000000000000000CF
:1001300000000000000000000000000000000000BF
:1001400000000000000000000000000000000000AF
:10015000000000000000000000000000000000009F
:10016000000000000000000000000000000000008F
:10017000000000000000000000000000000000007F
:10018000000000000000000000000000000000006F
:100190000933FF1F6931FF1FC16601000000000025
:1001A000000000000000000000000000000000004F
:1001B000000000000000000000000000000000003F
:1001C000000000000000000000000000000000002F
:1001D000000000000000000000000000000000001F
:1001E000000000000000000000000000000000000F
:1001F00000000000000000000000000000000000FF
:1002000000000000000000000000000000000000EE
:1002100000000000000000000000000000000000DE
:1002200000000000000000000000000000000000CE
:1002300000000000000000000000000000000000BE
:1002400000000000000000000000000000000000AE
:10025000000000000000000000000000000000009E
:10026000000000000000000000000000000000008E
:10027000000000000000000000000000000000007E
:10028000000000000000000000000000000000006E
:10029000000000000000000000000000000000005E
:1002A000000000000000000000000000000000004E
:1002B000000000000000000000000000000000003E
:1002C000000000000000000000000000000000002E
:1002D000000000000000000000000000000000001E
:1002E000000000000000000000000000000000000E
:1002F00000000000000000000000000000000000FE
:1003000000000000000000000000000000000000ED
:1003100000000000000000000000000000000000DD
:1003200000000000000000000000000000000000CD
:1003300000000000000000000000000000000000BD
:1003400000000000000000000000000000000000AD
:10035000000000000000000000000000000000009D
:10036000000000000000000000000000000000008D
:10037000F9B50011000000000000000000000000BE
:10038000000000000000000000000000000000006D
:10039000000000000000000000000000000000005D
:1003A000000000000000000000000000151BFF1FFF
:1003B000000000000000000000000000000000003D
:1003C000000000000000000000000000000000002D
:1003D000000000000000000000000000000000001D
:1003E000000000000000000000000000000000000D
:1003F00000000000000000000000000000000000FD
:081838000070FF1F4118FF1FA3
:10184000024981F3088802F063FB00000070FF1F6B
:1018500070B500241E491F4A1F484C6308CA1B0567
:101860001B0DE4188242F9D11C4B80228B630021AE
:1018700009201B4B920519621A4B1B4DDA671B4B53
:10188000DA688243DA609A68194802409A60112047
:10189000296002F095F8112002F072F86B6C154A7D
:1018A000112013406B64144B144A63431B0C1384C4
:1018B0000122134B9A7201F00DFC124B1B78002B86
:1018C00004D1114B1021187802F092FA70BDC04675
:1018D000000005408807054000080540FF010000A2
:1018E00000F0004004E100E0003800403CF000401F
:1018F000FFDFFFFFFFFDFFFFAE060000EC61FF1FF3
:10190000A062FF1FCE64FF1FCC62FF1F10B502F064
:1019100087F9072804D0122808D0022808D010BD63
:10192000044A0420136B01331363F8E70220F6E73F
:101930001420F4E7E065FF1FF8B507000C0026004F
:101940002500503630785135002804D10300287026
:1019500058342370F8BD2978CA00481E8141A31865
:101960003800A25C5B68C9B2FFF7D0FF00280DD138
:101970002B78DA00A218013350602B703378044AB8
:10198000013B3370136A01331362D8E70123DFE7A9
:10199000E065FF1F5C234343074910B5C9180B00DE
:1019A00058331B78012B05D1FFF7C6FF034A936A12
:1019B0000133936210BDC0461466FF1FE065FF1F30
:1019C00010B502F09DFB064A0121130010CB4942DD
:1019D000D967044B136002F0B3F9200010BDC04674
:1019E00000E100E01000100010B5040002F088FBD8
:1019F000024B1C6002F0A4F910BDC04600E100E0FB
:101A0000431E5A425341A022F0B5D2015B4213401B
:101A1000154D164A40019B182A18127E8BB0019171
:101A2000002A1BD01A000832D46F0022E6B206AF9B
:101A3000E4B294420EDC2818C369002B08D0019947
:101A400002AA117106AA049202AA167303A8984763
:101A50000BB0F0BD1978B9540132EAE71A7D1A7853
:101A600006AB01261A70E6E7A068FF1F00400040A1
:101A7000F0B5254B04004001C25C85B0002A2BD094
:101A80001A18117E002927D0917E002924D01179BF
:101A9000022921D11689D788D168F51BADB22A1C3D
:101AA000102D00D9102292B2BE4217D1181801236E
:101AB00003710023C269C38003819A4206D068463D
:101AC000032103730171029301A890470820002CA1
:101AD00000D0192001F0FEFA05B0F0BD013C6542CE
:101AE0006C41A0256442ED012C40084D1B1864197F
:101AF000074D0633013A92B2AA42EDD01888461C2F
:101B00001E80085C2070F5E7A068FF1F00400040C1
:101B1000FFFF00000F220E4B10B5986810400238EE
:101B20000A280BD802F060F80D0A0B0A0A110A0AFB
:101B30000A0A060002210020FFF762FF10BD012102
:101B4000F9E70020FFF794FFF8E7DB6FF6E7C04600
:101B5000004000400F220E4B10B59868104002382C
:101B60000A280BD802F040F80E0A0B0A0A120A0AD9
:101B70000A0A060002210120FFF742FF10BD0121E1
:101B80000800F9E70120FFF773FFF7E7DB6FF5E7E0
:101B90000090004013B5334C2378072B3DD8324BCF
:101BA0001A78324B002A39D18022196852020A432E
:101BB0001A60252001F0C4FE20232D4A11680B4332
:101BC000802113606B460422C90508680733104260
:101BD00028D080210422C905C86810422ED0802157
:101BE0002020C905CA688243CA6014221A701A7874
:101BF000002A2FD18021C905C86820320243CA605B
:101C000014221A701A78002A28D11A4B1A7D2278C9
:101C10005A601D221A705932DA6013BD1A681649CB
:101C20000A40C5E7086802430A6014221A701A784D
:101C3000002ACED01A78013AD2B2F7E7C868024338
:101C4000CA6014221A7019784A1ED2B21A7000297A
:101C5000F9D1C4E71A78013AD2B2C7E71A78013A43
:101C6000D2B2CEE72444FF1FEC44FF1F3CF00040FB
:101C70001C44FF1F00200040FFFFFEFF564B70B5C5
:101C80001B68012B03D1554A936D0133936502F014
:101C9000F7F9534B534A1860534B544C1A600123C5
:101CA000534A1360534A13602378002B06D0062250
:101CB0005149524801F0D4FF00232370504A514B40
:101CC00010681B78C1B2002B0ED14F4CC0B22378E4
:101CD0005BB2002B4FDB237824785BB264B21B0429
:101CE00024021B191B1813600B1C50294ED95023BA
:101CF000464A47491078DBB2FF2202284BD10868D8
:101D0000444C454D267890432A78964254D92278FF
:101D100024782E78023B5D10A31B6B435201D31A2B
:101D200010335B111843086001F0DAFF031F012B29
:101D300045D83A4B1B78002B06D0394B1B78002B2B
:101D400002D0002002F084F9A122364B920099784B
:101D5000354B4A431B689B18832292009B181B78C3
:101D6000033B012B03D8AF20400002F0A9F9012268
:101D70002E4BDA8270BD237824785BB264B2FF33D5
:101D8000FF341B0424021B190138ABE7CAB2022A34
:101D9000AED20223ACE70868254C264D2678904346
:101DA0002A78964208D9227824782D78023B5B1055
:101DB000641B63435201B2E72378DBB2B2E7022827
:101DC000D5D11D4B1B78013B022B03D91B4B1B7834
:101DD000022BCCD16C20C8E79809FF1FFC0FFF1F16
:101DE0001865FF1FFF3F0000141003401C65FF1F14
:101DF0000C10034000100340D50BFF1F7211FF1F92
:101E0000B40003408C09FF1F680AFF1F490AFF1F27
:101E100094000340460AFF1F470AFF1FF908FF1FEF
:101E20002209FF1F300DFF1F3409FF1FBC0BFF1FCE
:101E3000440AFF1F450AFF1F1C09FF1F2309FF1F3C
:101E400010B502F09DF80022014B1A8010BDC0466B
:101E50001665FF1F10B502F0ABF8A121054A8900F5
:101E60009478054A61431268044B5218528C1A80C8
:101E700010BDC046300DFF1F3409FF1F1665FF1F40
:101E800010B50D4B0D4A9978A1239B004B43126866
:101E9000D218531DD97F0A4B1B88994209D2441C82
:101EA00007D0C82805D0D2695B1A5A43054B534363
:101EB000C01801F075FF10BD300DFF1F3409FF1F62
:101EC0001665FF1F7102000070B5244D2B68002BB2
:101ED00028D001F09DFF2B68D8402B680400002B10
:101EE00027D001F0B5FE2B68D8401D4B1D4A9978CC
:101EF000A1239B004B431268D118D25C91239B0015
:101F0000002A20D0CA580132CA50174B17491B6803
:101F10000868834214D3D23B181A012A1AD0144BF2
:101F2000186070BD01F074FF124B196801F088FE53
:101F3000D3E701F08DFE0F4B196801F081FED4E765
:101F40000D495B18E8E7CA500C4B1B68DB68E418C6
:101F5000201AE4E7F530FF30E1E7C0461C08FF1F18
:101F6000300DFF1F3409FF1F9C09FF1F1865FF1F5D
:101F7000A009FF1F1808FF1F2DFF3F002065FF1F4E
:101F800070B504000D00282916D10300A433C288BF
:101F90001B889B1A0B4A9BB293420DD906006A36E6
:101FA00005223100653001F0BBFF002804D131006B
:101FB000200001F0B5FE70BD2900200001F030FFC7
:101FC000F9E7C046FE7F0000F8B50500012001F0EA
:101FD000FFFF134CA36AA26A9342FBD1114E3360F8
:101FE00001F0F6FE1049030008601048426894466C
:101FF0000F4A17680022BC4501D24268BA1A0D4840
:1020000002603268AD18A422E562606A520302439E
:102010006262094A1278002A01D00F3B0B60F8BDBA
:1020200000F00040340AFF1FE408FF1F28100040A2
:10203000180AFF1F1C0AFF1F1C09FF1F70B5802410
:102040001025E405A3682B43A36001F031FFA368CA
:10205000AB43A36070BD0000F7B5160080221C00E2
:102060001023D2050191916805000B439360002273
:102070005A4BD7301A6001F0DBFD9D232A002F0058
:102080009B00EB58CA3201210092FC37002B01D093
:102090000021009A386801F04BFE2900009BCB31EB
:1020A0001A784F4BD3351A604B780A781B021343CA
:1020B0008A7812041A43CB781B061343494A1BBA89
:1020C00013604B790A791B0213438A7912041A436D
:1020D000CB7931001B061343434A1BBA13606B785C
:1020E0002A781B021343AA7812041A43EB781B06C2
:1020F00013433E4A1BBA1360019A330213433C4A0E
:1021000013603C4B22001B1B9C4603293DDCB3089B
:102110009A0013005142B21A032A46D1354AE018F8
:10212000511A82784078120400020243E05C0433C2
:1021300002430A600022FF2B4BDDF0222E4B1201DE
:102140001A600F222D4B1A602D4A1368002BFCD009
:102150000023224A27491360091B321D0B191B68F3
:10216000043A180A23706070180C1B0EA070E370FC
:102170000434002AF2DC802210213B68D2050133AE
:102180003B6093688B439360F7BD6346D57898189E
:1021900093782D061B042B43157804392B4355786F
:1021A00004322D022B430360AFE7022A0AD1114A01
:1021B000E05C511AE2185278120202430A600433BA
:1021C0009BB2B7E7012AB5D10A4A521AE15C116005
:1021D000F5E7084959180A600433ACE700000440E9
:1021E0003C00044038000440340004403000044007
:1021F0000C000440000104400400044010000440AE
:1022000014000440F7B5150080221C001023D205ED
:102210000091916807000B4393600023654AD73013
:10222000136001F005FD9D233E009B00F9583B0023
:10223000CA363200FC33002900D07FE0586801F034
:1022400077FD390032785C4BCB311A604B780A78D5
:102250001B0213438A78AC4612041A43CB78281D1C
:102260001B061343554A1BBA13604B790A791B02AC
:1022700013438A7912041A43CB791B061343504A3D
:102280001BBA13604B7A0A7A1B0213438A7A120430
:102290001A43CB7A21001B0613434A4A1BBA136028
:1022A000009A2B021343484A13602200474B1B1B22
:1022B0000093009BCE785B1801938B7836061B0445
:1022C00033430E78043833434E78043136023343B7
:1022D000019E33600328ECDC0321A808431C9B000B
:1022E0002940800003292BD13849E5185E18A978C8
:1022F0006D78E35C09042D02294319433160030022
:1023000008330021FF2B2DDD314B324919600F219D
:10231000314B1960012327490B60304B19680029A4
:10232000FCD006211B680B40042B20D0802200200B
:10233000D20593680A318B439360FEBD01217DE78E
:10234000022908D121495D18E1184978E35C0902A6
:1023500019432960D3E70129D3D11C495918E35CFB
:102360000B60CCE71948181801600433CAE7002352
:1023700010490B606346002B0CDC3B00FC335A68B1
:10238000102101325A608022D205936801208B43CC
:102390009360D2E7009B9B181B68190A1370517059
:1023A000190C1B0ED37004235B4291709C440432C1
:1023B000E0E7C046000004403C0004403800044010
:1023C00034000440300004400C000440000104408C
:1023D00004000440080F00001000044014000440F2
:1023E00070B5061E19D002225A4B9B799343012BDC
:1023F00013D1594B1A78FF2A0FD15A78FF2A0CD1E2
:102400009A78FF2A09D1DA78FF2A06D11A79FF2AA9
:1024100003D15B79FF2B00D199E0504B0C201A7847
:10242000012A08D000224E4D1A7029780B00093B72
:10243000042B01D8212070BD4B1F012BFAD9454C2C
:10244000A37B042B00D982E0A279032A00D97EE085
:102450009A1ED2B2012A02D860881F2877D9002E8E
:1024600056D0012E73D1A0880128E3D0002907D1CE
:10247000581E032803D801F0B7FB121715122E704F
:102480002978481E032811D80025364B1D602823C3
:10249000237501F01DFCA84227D0A580CAE70221C0
:1024A0002970EDE70421FBE70321F9E7073901294A
:1024B000C0D82D490968C96A8906BBD52B49087857
:1024C0000028B7D1012A01D9002BB3D102230B7008
:1024D0008021274D263389012878237501F080FC5F
:1024E00080212878890101F083FC0123A380214BFE
:1024F0001B78002B0AD0FA2280211F4B92001B88E8
:1025000009025A431A4B187801F0F2FD002092E7B5
:1025100001F0F6FD2B78A680073B012B03D9174865
:102520002E7001F02DFC114B114C1A78002A06D0A8
:1025300080210022207889011A7001F051FC01F0FD
:10254000FFFB80212078090201F04AFCDEE712201F
:1025500071E7C046A60BFF1F6B09FF1F1A09FF1F7B
:102560001C09FF1F4809FF1F2065FF1F2309FF1FCC
:102570001B09FF1F2109FF1F2C09FF1F001000402E
:1025800010B5002901D001F0E3FB10BDF7B5604B99
:1025900001919978A1239B004B435E4A0600146881
:1025A0001022E418D6235B00E0583623FF33E35CA7
:1025B00000279343222B41D1574B0F3A1A600760F3
:1025C000012501F06DFC019B1880E8235B00E35CB2
:1025D000002B01D0B34258DD0023504FFB70AD33C8
:1025E000FF33E3581A68002A03D09B88DB439B071C
:1025F0001DD03823FF33E35C002B18D09B235B00F6
:10260000E35C002B13D1D133FF33E35CB3420EDA2A
:10261000A4235B00E15AE018090A023101F0F8FC3A
:1026200023000122FE33013E01351A87FA70E823A8
:102630005B00E35C002B2AD0A8B2FEBD03683D001E
:10264000002BBED081880430090A023101F0E0FC81
:10265000D6235B00E3581F60B2E72300B133BA0012
:10266000FF339858013781880430090A023101F09C
:10267000CFFCE8235B00E35CBB42EEDCE822F61A09
:10268000ED1800235200A354A6E70027F1E720002D
:1026900001F0B6FB00281FD0002E1DDD731988261F
:1026A00047190193B600200001F082FB5A308000E8
:1026B00020184068013581880430090A023101F090
:1026C000A7FC200001F0B4FBA3590133A351BD4284
:1026D00002D0019B9D42E6D1114BE35C002BABD0B5
:1026E00095239B00E35C002BA6D00E4BE15A0029FA
:1026F000A2D00D4AA35C994202D90133A3549BE7AF
:1027000000231A212000A35401F0C2FB94E7C04625
:10271000300DFF1F3409FF1F00140340E010FF1F9E
:102720005A020000720200005E0200000D4970B5FE
:102730004A6E0D4CD2038B69D20BA24206D80B4DC8
:102740000224AA4204D901F0ABFC70BD0224644209
:10275000E21815007E2425402242F4D0A3432B43E7
:102760008B61F0E700F000400A200000FC1C000034
:10277000F8B51D4B1D4F1A78002A10D1BA7B002ADC
:1027800002D101321A7003E0032AFAD0022AF8D0EB
:1027900001F09EFA00220120154B1A70F8BD154B6E
:1027A000154D1C68154B9E7801232B702878C0B2FC
:1027B00000F0A2FBBB7B002B0BD101F081FAA1231F
:1027C0009B007343E41883239B00E41823782B7049
:1027D000E4E7032B02D101F083FBF0E70020022B9A
:1027E000DCD101F015FAEAE71C09FF1FA60BFF1F59
:1027F0002309FF1F3409FF1F490AFF1F300DFF1F68
:10280000F0B587B00EAD2F780FAD2D780593AC469F
:10281000634614000E4D0CAA12782E7803930D9B7C
:10282000009201932200059B029701F051FB2E704C
:10283000012C01D0042C08D1802206498B889343B7
:10284000054A1278D20113438B8007B0F0BDC04611
:102850001C09FF1F6C11FF1F7809FF1F0B001B3B9A
:1028600070B504003020E02B0DD81300E025493B63
:10287000FF3B9BB2ED00AB4205D8034B2000198211
:102880005A8201F0EDFA70BD8410FF1F10B501F0FF
:10289000F7FB054B00205B68052B04D9034A5268FF
:1028A000D20200D4980810BD00100040FCE100E006
:1028B00070B501F025FC0D4B1B68FC33DC691D6A0B
:1028C000FFF7E4FF6419844204D2094B01241B681A
:1028D000002B07D004220024064B1A70064A936985
:1028E0000133936101F02CFA200070BD2065FF1FB9
:1028F0009809FF1F2309FF1FFC0FFF1F70B50C4D28
:102900002B68FC335C6A01F0FBFBFFF7BFFF2B6811
:102910000025FC339B6AE318834204D2054B1B68F5
:10292000AB4200D1051B01F00BFA280070BDC04678
:102930002065FF1F9809FF1FD722044B92009B5868
:1029400010B5002B00D0984710BDC0460000FF1FF7
:1029500010B501F0D3F8FFF7EFFF2749274BCA6DF9
:10296000274C1A4084235B001343CB65254B1B681F
:10297000186A01F02DFB244B244A1A60244B254A87
:102980001A60A022244B52001A60244B187801F0E0
:1029900027FB2000224901F06BFA0023A3600233D9
:1029A000A360204B2049236003232048A36001F04B
:1029B0005FFA10221E4BFF201A60802252031A6019
:1029C000802292031A60802212041A6001F040FBF8
:1029D000012001F0F5F9FA20400001F0B1FA582089
:1029E00001F06EFB134801F083F9012001F050F96A
:1029F000072001F005FB10BD00F0004000FEFEFFC7
:102A0000141000402065FF1F000003400180063DB8
:102A1000BC00034034080000A40003404A0AFF1F22
:102A200071020000C3090000FFFF3F0028100040B2
:102A300000E100E030750000674E336888331B68A2
:102A400083F3088801F084FA644A6549136800201A
:102A50000B401360634B644A1B68934200D1A6E0AD
:102A600001F026F90221614A13688B431360FFF7D6
:102A70006FFF5F4B5F4C1878C0B201F029FB002359
:102A8000A3600233A3605C4B0120236001F0A0FA35
:102A90000323A36001F07CFA040001F0F1FA0500C1
:102AA00001F076FA554B186001F022FA544B196880
:102AB000621A531EA14200D213008022D203934215
:102AC00001D39B029B0A3268D16AC90700D471E026
:102AD0004C491C0C09689BB24C4359432402090A17
:102AE000641803264849FC3293680A6847489B1AD1
:102AF000474A0768126847499B18474A9A18334063
:102B00009208DB190A600360042B03D901323340B9
:102B10000A6003600E684149A619300001F090F880
:102B20003F4F3E493B68C3183B603000019301F0C2
:102B3000FFF93C4E3068081838493060884205D9A2
:102B4000019B01333B6001F0F3F9316001F0E0FAE1
:102B5000354B1B78002B0DD001F092FA334B621BE2
:102B6000196812188A4232D24919091B091A3048C9
:102B700001F07EF92F4E337A002B0ED001F080FA4F
:102B8000621BF1681218914224D94919091B091ACC
:102B9000294801F06DF900233372284B83F308882C
:102BA00001F056F9002001F083F801F079F801F006
:102BB0007FF85CE7DC0199000234641A5900641A5A
:102BC00009214B438033CB40A408E41889E7FA215C
:102BD0008900CCE71A49DBE72065FF1F1CF00040A5
:102BE000FFFFC1FF0C0AFF1FB64121031000004088
:102BF000490AFF1F14100040C3090000100AFF1FFC
:102C0000340AFF1F380AFF1F200AFF1F280AFF1F70
:102C10001C0AFF1F240AFF1FC409000071020000E4
:102C20006008FF1F2C0AFF1F1C09FF1FE408FF1F7D
:102C300000100040740BFF1F3C10004000000020FB
:102C4000DC050000A022054B92009B5810B5002B1C
:102C500001D0984710BD01F02BFAFBE70000FF1FE1
:102C6000A122054B92009B5810B5002B01D098472C
:102C700010BD01F01DFAFBE70000FF1FA222054B6B
:102C800092009B5810B5002B01D0984710BD01F061
:102C90000FFAFBE70000FF1FA322054B92009B5891
:102CA00010B5002B01D0984710BD01F001FAFBE7E9
:102CB0000000FF1FA422054B92009B5810B5002B6B
:102CC00001D0984710BD01F0F3F9FBE70000FF1FAA
:102CD00070B501F0D5F94F4B186001F0D1F8040040
:102CE000C30702D401F044F970BD00224A4B1A60B8
:102CF0004A4B18780138042829D800F075FF0320C2
:102D0000181C2400200000F0B3FF0128ECD0444C34
:102D10002378042B6ED101F053F90028E4D001F0A0
:102D2000A7F9582001F0CCF902232370DCE720003A
:102D300001F0AEF9E9E7200001F082F8E5E72000B4
:102D400001F08EF9E1E7200001F02AF9DDE700F05B
:102D5000C7FF0500012808D1324B1B78053B012B2A
:102D600003D82000FFF76EFFD1E72D4B1B78022B15
:102D700001D0052B20D1022D28D12B4B9B7BAB43BF
:102D80001CD12000FFF76CFF264B18780128BED11C
:102D90006405BCD4244925224B7B034205D1233A48
:102DA00013405A42534126331A000B7D9342AED949
:102DB000322001F03DF9AAE7022D07D1194B1B780B
:102DC000052B11D12000FFF759FFDDE7012D0BD1B5
:102DD000012B03D12000FFF75FFF98E7062B03D1FB
:102DE0002000FFF767FF92E7200001F061F9022D54
:102DF0008DD1C9E7032B04D10C4B987C01F060F80E
:102E000072E7072B00D06FE7094B987B00F0A8FF13
:102E10006AE7C0469C09FF1F9809FF1F9009FF1F22
:102E20002309FF1F1C09FF1FA60BFF1FBC0BFF1F61
:102E3000D40BFF1FFA210A4B0A4A49001A640A4AB6
:102E40005A500A4A04395A50094A08319A64094AC0
:102E50005A50094A5C315A50084ADA667047C046EF
:102E60000000FF1F0128FF1FFD28FF1FB128FF1FC3
:102E7000E123FF1F7127FF1F811EFF1F551EFF1F2C
:102E800010B500F099FE10BDF7B50B0CFF2701221D
:102E9000009300233C001E001D009446019089B25F
:102EA00062469A401000084018413618B6B2FF2F0B
:102EB00002D1012E00D19FB2009802401A41AD18F4
:102EC000ADB2FF2C02D1012D00D19CB20133102BE9
:102ED000E6D10320012E07D1012D04D1019B24014D
:102EE000E4191C700138FEBD102EFCD10238102DE3
:102EF000F9D00230F7E700008023F7B59C46264B57
:102F0000264F01932649274A274D284C284B022853
:102F10001AD1604638600868264E30408026360355
:102F20003043086001990978002909D11660224AC6
:102F30002A60224A2260E02219689143A03A1BE0ED
:102F40008021C9021160F2E766463E600F68194EA3
:102F50003E408027FF023E430E6001990978002918
:102F60000DD1176001280ED1154A2A60154A22603A
:102F7000E02219689143C03A0A431A60F7BD8021E4
:102F800089021160EEE7E0210F4A02432A600F4AEE
:102F900022601A688A43F0E74B0AFF1FE0000340F3
:102FA000D80003409000034000000340500003405D
:102FB00040000340FFFFE3FF0280063D80450822FA
:102FC0000180063D80660822008006988055082210
:102FD000F8B51E4B80261A68002014003440324297
:102FE00032D11A681A4F32431A6001223B68063008
:102FF00093433B6000F0ECFF0122164D2B681E430B
:103000002E603B680A2613433B608027BF00124BAB
:103010001B683B4211D1013EF6B2FF2E09D17E2240
:103020000E4B1C682B68E40B1440934323432B6026
:1030300005E0082000F0CCFFE9E7002EEFD1802268
:103040002B68600893432B60F8BDC046C4F0004075
:103050005CF0004018F0004068F0004060F0004074
:1030600010B500F04DFF01215820034A00F0E8FFA1
:10307000FFF7AEFF10BDC046600AFF1F10B57822F3
:103080000021034801F02CF800F0CAFF002010BD19
:103090002868FF1F70B5040001F032F800230C20EF
:1030A0000B4A010059438D18515C00290DD0A142F3
:1030B00008D1012300246B7000F06AFE00F040FE8E
:1030C000200070BD01330A2BEBD11224F6E7C04675
:1030D0002868FF1F70B5040001F012F800231900E2
:1030E0001D000D4A1078002806D0A0420CD1557062
:1030F00001310C320A29F5D1002B0AD100F090FFE2
:1031000000F01EFE002070BD5078461EB0411B1816
:10311000EEE700F03DFEF3E72868FF1FF7B5040077
:103120000C20002384460E4D019267465F43E85D04
:103130007E19A04212D000280BD10A4B9C46624651
:103140001B7808331370019B70707C557160B360FD
:10315000FEBD01330A2BE8D10320F9E70720F7E78A
:103160002868FF1F2468FF1F8020F8B5484BC00562
:103170001B68C1248360474BFF251A680123134352
:103180004361454BA4001A68444B40211A60444BEC
:103190001A68444B1A60444B1A59AA431A51C52263
:1031A00092009E58AE433143802699509F583F4924
:1031B000F6010F403E439E509E5880273602360A45
:1031C0003043985080201A5900020A4002431A5195
:1031D00004341A59364E3F04324080263A431A517D
:1031E0001A5936061202120A32431A5108341A5971
:1031F00080260A4002431A51C32292009F58B446C7
:10320000AF4337439F509F58294E0F4007439F506D
:103210009F58374080263604374380269F509F585A
:1032200036063F023F0A37439F50C0221F59AF4323
:103230003A431A511A591202120A1643C6221E5153
:1032400092009C58AC4365462C439C509C580025EA
:103250000C4020439850C72080001A58154C11404C
:10326000C02212020A431A50134B1B78DB08AB42F0
:1032700001DC0020F8BD2378002B06D0A368002BCA
:1032800000D0984701350C34EEE71220F2E7C04633
:103290002044FF1F1C44FF1FB0F000402068FF1FA8
:1032A000B4F000401C68FF1F00E100E0FF00FFFFDA
:1032B000FFFF00FF2868FF1F2468FF1F030010B5F1
:1032C0001F2809D8072200201340072404490A7840
:1032D000A24313430B7010BD00230620F5E7C04640
:1032E0002468FF1F054B06491B780A6805485B07E1
:1032F00002401B0B134300200B6070472468FF1F24
:103300001CF00040FFFFC1FF70B50C25FFF7EAFF7E
:103310000A4B1C780A4BE4086543ED18002C01D1D8
:10332000200070BD2B78002B06D06B68002B00D0DE
:103330009847013C0C3DF1E71220F2E72468FF1F9B
:103340001C68FF1F1FB5002102220B000191009194
:10335000052000F00DFD02230B490A681A42FCD13A
:1033600020230393039B5A1E0392002BFAD1074A92
:103370001368002BFCDA0B246C442000012100F0C0
:10338000C7FC207804B010BD90C8004000C80040C1
:1033900013B504000A4B0193019B002B01D11120AE
:1033A00016BDFFF7CFFF23000340044205D00520E0
:1033B00000F00EFE019B013BEDE71800F0E7C04670
:1033C000FFFFFF0707B500F09BFE80220821D20512
:1033D000936A0191002B01D10739916202210C4AB5
:1033E00011600199481E01900029FAD10331116042
:1033F000053101910199481E01900029FAD111600F
:10340000002B02D18022D205936200F099FC07BD07
:1034100000C00040F0B52D4C89B02378002B4FD16F
:10342000FEF7CEFA02232A4F03903A681A42FCD1E3
:1034300020230693069B5A1E0692002BFAD1254E96
:103440003368002BFCDA0120FFF7A2FF011E02D037
:10345000112009B0F0BD030003220190009005ADDA
:103460009F2000F085FC0321280000F051FC02237E
:103470003A681A42FCD120230793079B5A1E0792F1
:10348000002BFAD13368002BFCDA0120FFF780FF14
:103490000028DDD10398FEF7A7FAAA786B7811040B
:1034A0001B020B4329780B4363601300113B0A494D
:1034B000052B07D801239340A3600B6001232370E1
:1034C0000020C6E780231B03F6E7C0460844FF1F21
:1034D00090C8004000C800409808FF1F1E4B30B540
:1034E0005A6818781D4B85B0D31859424B410121B9
:1034F0000093002300F004FC194B1A4A02259A633A
:1035000000221A6510325A658022C4219D65164B2F
:103510001648D202DA6789004258154B80241A40B7
:1035200080231B0413434350642341200393E40589
:1035300000F006FA402000F003FA6562039D6B1E5E
:103540000393002DFAD103236362FFF73BFFA562CB
:10355000FFF760FF05B030BD1444FF1F95FFFEF775
:1035600000C80040050001FF04E100E000E100E0C8
:10357000FFFF00FFF0B585B00700FEF721FA022338
:1035800005002D4C22681A42FCD120230093009B99
:103590005A1E0092002BFAD1284E3368002BFCDA19
:1035A0000120FFF7F5FE002803D01124200005B00C
:1035B000F0BD234B2360022322681A42FCD1202352
:1035C0000193019B5A1E0192002BFAD13368002B04
:1035D000FCDA0120FFF7DCFE0028E6D1194B1F6062
:1035E000022322681A42FCD120230293029B5A1E16
:1035F0000292002BFAD13368002BFCDA0120FFF78E
:10360000C7FE0028D1D1104B2360022322681A4242
:10361000FCD120230393039B5A1E0392002BFAD163
:103620003368002BFCDA0120FFF7B2FE041EBCD188
:103630002800FEF7D9F9B9E790C8004000C800405B
:1036400001000006A8C800400180000110B500205C
:10365000FFF790FF10BD000010B5064B18705960C1
:10366000FFF73CFF00211320034AFFF757FD00201E
:1036700010BDC0461444FF1FDD34FF1FF0B5040029
:1036800085B003920291FEF79BF9882263035B0BDE
:1036900052051A438023DB059D6A8023274F009241
:1036A000BA68002601901B039A420CD9F823260021
:1036B0001B041E401C4206D08022214B52025E6237
:1036C00019680A431A60002D0BD100F019FD02227F
:1036D0001C4B1A608023DB055A62013A9A6200F0A3
:1036E0002FFB0023039A934220D1002D0AD100F032
:1036F00007FD144B03221D608023DB055A629D6287
:1037000000F01EFB8023BA681B039A4208D9002EE2
:1037100006D000220A4B0C495A621A680A401A6005
:103720000198FEF761F9002005B0F0BD009A0299FA
:10373000D2181278CA540133D4E7C0460844FF1F98
:1037400000C8004000C00040FFFFFEFFF0B587B09A
:10375000029103920400FEF733F9019000F0D0FCCF
:10376000802302250122234EDB0535605D629A62CB
:1037700000F0E6FA204F3B682B42FCD12023049353
:10378000049B5A1E0492002BFAD11C4D2B68002B6F
:10379000FCDA0120FFF7FCFD002802D0112007B061
:1037A000F0BD2000039A029900F022FC02230400DD
:1037B0003A681A42FCD120230593059B5A1E0592B4
:1037C000002BFAD12B68002BFCDA0120FFF7E0FD7B
:1037D000051EE3D100F094FC80230322DB05356055
:1037E0005A629D6200F0ACFA0198FEF7FDF8E0B273
:1037F000D5E7C04600C0004090C8004000C8004067
:10380000F0B5802489B00600FEF7DAF8E405A36A73
:1038100002250393029000F073FC0123304F3D60BA
:103820006562A36200F08CFA2E4C23682B42FCD117
:1038300020230593059B5A1E0592002BFAD12A4D91
:103840002B68002BFCDA0120FFF7A2FD002803D033
:103850001124200009B0F0BD244B2360022322680C
:103860001A42FCD120230693069B5A1E0692002B77
:10387000FAD12B68002BFCDA0120FFF789FD021E2C
:10388000E6D11B4B03211E60030001900090202015
:1038900000F06EFA022322681A42FCD1202307931B
:1038A000079B5A1E0792002BFAD12B68002BFCDADB
:1038B0000320FFF76DFD041ECAD100F021FC802318
:1038C0000322DB053C605A629C6200F039FA039BDC
:1038D000002B01D1FFF776FD0298FEF785F8B8E7D7
:1038E00000C0004090C8004000C800400100000631
:1038F00094C8004007B5000201910422000A01A902
:10390000FFF724FF0EBD000073B5050005240B4A28
:10391000A3005B429B1819686B46DE1D3000FFF761
:10392000B3FA022804D133782B55013CEFD276BD8F
:10393000052CFCD00128FAD10230F8E71409001157
:103940001F2807D8012380228340D20591680B43AA
:10395000936070473F2808D8012380222038834095
:10396000D20551690B435361F3E75F28F1D8012376
:10397000802240388340D205116A0B431362E8E786
:103980001F2807D8012280218240C9058B689343F4
:103990008B6070473F2808D8012280212038824060
:1039A000C9054B6993434B61F3E75F28F1D80122C6
:1039B000802140388240C9050B6A93430B62E8E7D7
:1039C0001F2810D880230200DB05153A1968012A48
:1039D00006D820229143196019680A431A6070477B
:1039E00001228240F6E73F2811D880230200DB0540
:1039F000353AD968032A06D810229143D960D9688C
:103A00000A43DA60EBE7012220388240F5E75F28BD
:103A1000E5D842238022181A413B8340D205516ADF
:103A200099435162516A0B435362D8E710B50400C1
:103A3000012813D1A022184992050B685B015B098C
:103A400013430B60154B164A19681140154A0A4377
:103A50001A60402219680A431A6010BD0028FCD180
:103A600001000A2000F07CFA21000B2000F078FA17
:103A7000C0220A4B920019680A4340211A601A6852
:103A80008A431A60B022044912060B685B015B0985
:103A900013430B60E1E7C04614F000401CF0004007
:103AA0007F00FEFF80FD010072B6074A13680133F4
:103AB00013600422054B1A600023054A136080221C
:103AC000D2055360FEE7C0467808FF1FC0F00040F3
:103AD000C4F0004005490B68002B05D1044A0A6078
:103AE00004490A60044A13607047C046140AFF1F65
:103AF000841E0000380AFF1FC4F000400023034A60
:103B00001360034A1360034A1360704754F0004087
:103B100040F1004044F10040002310B5184C8AB039
:103B2000009301932378012B27D06946012000F0F0
:103B3000A7F8002817D1009B12490293019B06AAFF
:103B40000393114B02A81B680493104B1B68059349
:103B500000F0AEF910220E4906A800F0E1F90028A5
:103B600004D1FF23237000200AB010BD0123094AAD
:103B7000074902A8237000F09BF90120F4E7C04632
:103B80002465FF1F10290011082900110C290011BC
:103B9000202900112865FF1F13B501246946012063
:103BA00000F06EF8034B00940193FFF7B5FF20007F
:103BB00016BDC046BB0B000010B5FFF79FFFFFF717
:103BC000EBFF002802D0024B984710BDFEE7C0462D
:103BD000E1A2000002B471464908490009564900B3
:103BE0008E4402BC7047C04602B471464908490081
:103BF000095C49008E4402BC7047C04603B471465C
:103C0000490840004900095A49008E4403BC7047E6
:103C100001B40248844601BC604700BF19FA0000A5
:103C200001B40248844601BC604700BFE927000098
:103C300001B40248844601BC604700BF89440000CB
:103C400001B40248844601BC604700BF090E000071
:103C500001B40248844601BC604700BF6D0B0100FF
:103C600001B40248844601BC604700BFE94C010032
:103C700001B40248844601BC604700BF0134010022
:103C800001B40248844601BC604700BFE1AC0000BB
:103C900001B40248844601BC604700BFE512010040
:103CA00001B40248844601BC604700BF8552010050
:103CB00001B40248844601BC604700BF016C0100AA
:103CC00001B40248844601BC604700BFE9F6000029
:103CD00001B40248844601BC604700BFA9D8000077
:103CE00001B40248844601BC604700BFDD0C0100FE
:103CF00001B40248844601BC604700BF8D11010039
:103D000001B40248844601BC604700BFC56D010094
:103D100001B40248844601BC604700BF3D71010008
:103D200001B40248844601BC604700BF85C1000061
:103D300001B40248844601BC604700BF2144000032
:103D400001B40248844601BC604700BF9DA9000041
:103D500001B40248844601BC604700BFE9D40000BA
:103D600001B40248844601BC604700BFC1F70000AF
:103D700001B40248844601BC604700BF496D0100A0
:103D800001B40248844601BC604700BFC1A50000E1
:103D900001B40248844601BC604700BF21A900006D
:103DA00001B40248844601BC604700BF8937010066
:103DB00001B40248844601BC604700BFD9B000008E
:103DC00001B40248844601BC604700BF691101008C
:103DD00001B40248844601BC604700BFBD5C0100DD
:103DE00001B40248844601BC604700BFB3520100E1
:103DF00001B40248844601BC604700BF0D52010077
:103E000001B40248844601BC604700BF71B00000A5
:103E100001B40248844601BC604700BFE90B0100C1
:103E200001B40248844601BC604700BF51B800009D
:103E300001B40248844601BC604700BF59760100C6
:103E400001B40248844601BC604700BF053401004C
:103E500001B40248844601BC604700BF7997000066
:103E600001B40248844601BC604700BF116E0000E7
:103E700001B40248844601BC604700BF2D6C0100BC
:103E800001B40248844601BC604700BFBD0B01007D
:103E900001B40248844601BC604700BF53B900002A
:103EA00001B40248844601BC604700BFCD0C01004C
:103EB00001B40248844601BC604700BFDD3F0000FA
:103EC00001B40248844601BC604700BF4DF90000C0
:103ED00001B40248844601BC604700BF9D6A0000EF
:103EE00001B40248844601BC604700BF75F8000079
:103EF00001B40248844601BC604700BFC1660100AE
:103F000001B40248844601BC604700BFED6801006F
:103F100001B40248844601BC604700BF01B60011ED
:103F200001B40248844601BC604700BFCD4C01008B
:103F300001B40248844601BC604700BF090E00007E
:103F400001B40248844601BC604700BF85120100ED
:103F500001B40248844601BC604700BFC9A9000003
:103F600001B40248844601BC604700BF7DA2001135
:103F700001B40248844601BC604700BFDD0A01006D
:103F800001B40248844601BC604700BF8D82000036
:103F900001B40248844601BC604700BF156B0100B4
:103FA00001B40248844601BC604700BFF9350100F6
:103FB00001B40248844601BC604700BFF9ED00002F
:103FC00001B40248844601BC604700BF01D700002D
:103FD00001B40248844601BC604700BF018900006B
:103FE00001B40248844601BC604700BFEDA5000053
:103FF00001B40248844601BC604700BF95730100CC
:1040000001B40248844601BC604700BFF90D0100BD
:1040100001B40248844601BC604700BFC1150100DD
:1040200001B40248844601BC604700BFADAE000049
:1040300001B40248844601BC604700BF61370100FB
:1040400001B40248844601BC604700BF016701001B
:1040500001B40248844601BC604700BFED6B01001B
:1040600001B40248844601BC604700BFF535010039
:1040700001B40248844601BC604700BF6DF60000F1
:1040800001B40248844601BC604700BFC95C01001E
:1040900001B40248844601BC604700BF09340100F6
:1040A00001B40248844601BC604700BFD1AE0000A5
:1040B00001B40248844601BC604700BFE917010013
:1040C00001B40248844601BC604700BF7912010078
:1040D00001B40248844601BC604700BF8914010056
:1040E00001B40248844601BC604700BFB70E00001F
:1040F00001B40248844601BC604700BF8B520100F6
:1041000001B40248844601BC604700BF75A90000A5
:1041100001B40248844601BC604700BFD544010099
:1041200002000000CABE001101000000B8BC00116E
:1041300002000000C6BE0011010000006041FF1F28
:1041400002000000C0BC0011010000009C62FF1FC3
:1041500002000000C4BE0011030000001062FF1F37
:104160001200000002000000CABE001101000000A1
:1041700000BD001102000000C6BE001101000000D9
:10418000FDBC0011020000000ABD00110300000088
:104190004B62FF1F02000000C4BE001103000000BC
:1041A0006062FF1F02000000C6BE00110100000097
:1041B000FCBC00110200000008BD0011030000005B
:1041C0002162FF1F02000000C4BE001103000000B6
:1041D0004262FF1F02000000CABE00110100000081
:1041E00044BD001102000000C6BE00110100000025
:1041F000A942FF1F0200000056BD0011010000008F
:104200003BBD001102000000C6BE0011010000000D
:10421000A842FF1F0200000054BD00110100000071
:104220006862FF1F02000000C6BE0011010000000E
:10423000A742FF1F0200000052BD00110100000054
:104240002BBD001102000000C6BE001101000000DD
:10425000A642FF1F0200000050BD00110100000037
:1042600026BD001102000000C6BE001101000000C2
:10427000A542FF1F020000004EBD0011010000001A
:1042800021BD001102000000C6BE001101000000A7
:10429000A442FF1F020000004CBD001101000000FD
:1042A0001CBD001102020202020200000000000018
:1042B000141300009D4B0011634B001198BD0011B9
:1042C00090011D0018001800FFFF070102030405FC
:1042D00006020106000000000000000000000000CF
:1042E00000000000000000000000000000000000CE
:1042F0000300000002000000CABE0011010000001F
:10430000B8BD001102000000C6BE0011010000008F
:104310006443FF1F02000000C2BD00110100000045
:104320009662FF1F02000000C4BE001103000000DF
:104330000065FF1F02000000C6BE00110100000062
:104340006443FF1F02000000C0BD00110100000017
:104350009862FF1F02000000C4BE001103000000AD
:10436000F864FF1F12006C6C0000000000000000E9
:10437000000000000807000000010000000001111B
:10438000FFFF000050485936000000000000000008
:104390000B000500F0000000B400002800280028F1
:1043A0003075A000A000A000A00000080008E001F7
:1043B000F00010001000100010001000100050005D
:1043C0005000500010001000D00700000000000056
:1043D0000F0001000500307507001000010081FF8B
:1043E00000000000FF000000657400116D720011F4
:1043F000FD6F0011FFFF0100FF000000819E001112
:10440000FD9B0011159B0011000000000000000042
:1044100000000800040000003B0001085902E00110
:1044200088212800FF00000002000000CABE001121
:104430000100000090BF001102000000C6BE001184
:1044400001000000A544FF1F02000000C2BE0011D1
:1044500001000000E068FF1F02000000C6BE00115E
:1044600001000000A444FF1F02000000C0BE0011B4
:1044700001000000A244FF1F02000000C6BE0011A0
:1044800001000000A044FF1F02000000BEBE00119A
:10449000010000009844FF1F180018001D00900143
:1044A000020000030202000002000000CABE001168
:1044B00001000000A4BF001102000000C6BE0011F0
:1044C00001000000E844FF1F02000000BCBE001114
:1044D000000000000000000002000000C4BE001147
:0A44E000030000000069FF1F20FF29
:040000051FFF184180
:00000001FF
